:100000000C9483000C94C2180C949B180C94AB00B5
:100010000C94AB000C94AB000C94AB000C94AB00B4
:100020000C94AB000C94AB000C94AB000C94AB00A4
:100030000C94AB000C94601A0C94AB000C94AB00C5
:100040000C9451180C94AB000C940F190C94E918F3
:100050000C94AB000C94AB000C94AB000C94AB0074
:100060000C9441190C94AB002A0042504D3A0054B4
:10007000617000202020202020202020202020200F
:10008000202020005265616479205B76312E395D35
:10009000005265616479205B76312E395D2A00203B
:1000A0007365740053746570200000000000240024
:1000B00027002A0000000000250028002B00000077
:1000C000000023002600290004040404040404049E
:1000D00002020202020203030303030301020408F3
:1000E00010204080010204081020010204081020A2
:1000F00000000008000201000003040700000000E7
:1001000000000000871A11241FBECFEFD8E0DEBF29
:10011000CDBF13E0A0E0B1E0E2E2F9E602C0059055
:100120000D92AE3DB107D9F726E0AEEDB3E001C0C8
:100130001D92A73FB207E1F710E0C3E8D0E004C08A
:100140002197FE010E945F33C238D107C9F70E9490
:10015000991B0C948F340C940000833081F028F4A8
:10016000813099F08230A9F008958730A9F0883065
:10017000C9F08430B1F4809180008F7D03C08091FC
:1001800080008F7780938000089584B58F7784BD39
:10019000089584B58F7DFBCF8091B0008F778093D9
:1001A000B00008958091B0008F7DF9CFCF93DF9399
:1001B000282F30E0F901E051FF4F8491F901E4521A
:1001C000FF4FD491F901E853FF4FC491CC23A1F024
:1001D00081110E94AD00EC2FF0E0EE0FFF1FE25402
:1001E000FF4FA591B491EC91ED2381E090E009F4EB
:1001F00080E0DF91CF91089580E090E0FACF1F93E7
:10020000CF93DF93282F30E0F901E051FF4F849125
:10021000F901E452FF4FD491F901E853FF4FC49123
:10022000CC23A9F0162F81110E94AD00EC2FF0E035
:10023000EE0FFF1FEC54FF4FA591B4918FB7F894C8
:10024000EC91111108C0D095DE23DC938FBFDF91B4
:10025000CF911F910895DE2BF8CFCF93DF9390E0DD
:10026000FC01E452FF4F249188539F4FFC0184917D
:100270008823C9F090E0880F991FFC01E655FF4FD5
:10028000A591B491FC01EC54FF4FC591D49161113B
:100290000DC09FB7F8948C91209582238C93888110
:1002A000282328839FBFDF91CF910895623051F4B6
:1002B0009FB7F8943C91822F809583238C93E8819B
:1002C0002E2BEFCF8FB7F894EC912E2B2C938FBF62
:1002D000EACF8E50806480937C0080917A008064A5
:1002E00080937A0080917A0086FDFCCF809178001F
:1002F0009091790008953FB7F89480918A05909184
:100300008B05A0918C05B0918D0526B5A89B05C0E5
:100310002F3F19F00196A11DB11D3FBFBA2FA92F84
:10032000982F8827BC01CD01620F711D811D911D81
:1003300042E0660F771F881F991F4A95D1F70895ED
:100340008F929F92AF92BF92CF92DF92EF92FF92E5
:100350004B015C010E947B016B017C010E947B01CF
:100360006C197D098E099F09683E734081059105CE
:10037000A8F321E0821A9108A108B10888EEC80EFE
:1003800083E0D81EE11CF11C81149104A104B10486
:1003900029F7FF90EF90DF90CF90BF90AF909F90A4
:1003A0008F9008952FB7F894609186057091870516
:1003B00080918805909189052FBF0895089508952B
:1003C0000895AF92BF92CF92DF92EF92FF920F9378
:1003D0001F93CF93DF936C017B018B01040F151FDB
:1003E000EB015E01AE18BF08C017D10759F0699143
:1003F000D601ED91FC910190F081E02DC6010995A7
:10040000892B79F7C501DF91CF911F910F91FF9053
:10041000EF90DF90CF90BF90AF900895FC01538D87
:10042000448D252F30E0842F90E0821B930B5417CE
:1004300010F0CF96089501970895FC01918D828D5B
:10044000981761F0A28DAE0FBF2FB11D5D968C91F4
:10045000928D9F5F9F73928F90E008958FEF9FEF33
:100460000895FC01918D828D981731F0828DE80FEF
:10047000F11D858D90E008958FEF9FEF0895FC01A9
:10048000918D228D892F90E0805C9F4F821B910976
:100490008F739927089588E496E00E943F0221E037
:1004A000892B09F420E0822F089580E090E0892BC9
:1004B00029F00E944B0281110C9400000895FC0168
:1004C000A48DA80FB92FB11DA35ABF4F2C91848DB5
:1004D00090E001968F739927848FA689B7892C9312
:1004E000A089B1898C91837080648C93938D848D65
:1004F000981306C00288F389E02D80818F7D808368
:100500000895EF92FF920F931F93CF93DF93EC0127
:1005100081E0888F9B8D8C8D98131AC0E889F989AA
:10052000808185FF15C09FB7F894EE89FF896083AD
:10053000E889F98980818370806480839FBF81E02E
:1005400090E0DF91CF911F910F91FF90EF90089570
:10055000F62E0B8D10E00F5F1F4F0F731127E02E4B
:100560008C8D8E110CC00FB607FCFACFE889F98983
:10057000808185FFF5CFCE010E945F02F1CFEB8D28
:10058000EC0FFD2FF11DE35AFF4FF0829FB7F89457
:100590000B8FEA89FB8980818062CFCFCF93DF9375
:1005A000EC01888D8823B9F0AA89BB89E889F9898B
:1005B0008C9185FD03C0808186FD0DC00FB607FCC0
:1005C000F7CF8C9185FFF2CF808185FFEDCFCE01F3
:1005D0000E945F02E9CFDF91CF91089520916C04D2
:1005E000260F3327331F21323105ECF42091B40557
:1005F000FC0190E080E0243069F082E00895A09151
:100600006C042191AC01445B5B4FA40FB52FB11D6D
:100610002C930196861798F380916C04680F609371
:100620006C0480E0089581E008951092B40581E0A3
:100630008093B30510928E0561E082E10E94FF0075
:1006400061E083E10E94FF00E9EBF0E080818E7FB2
:10065000808380818D7F808388E48093B80085E4E7
:100660008093BC000895CF93DF9391E090934B0467
:100670008823B9F0C091B800D091BA008091BC0035
:100680008A7B8093BC0060E082E10E94FF0060E012
:1006900083E10E94FF000E941503D093BA00C0932B
:1006A000B800DF91CF9108958F929F92AF92BF9241
:1006B000CF92DF92EF92FF920F931F93CF93DF932E
:1006C000D091DD05D13208F0D7C0182FC091DC05DC
:1006D0000E947B016B017C018091B40581116BC08C
:1006E00082E08093B4051093B3058FEF8093B20539
:1006F0001092B105D093B005ACEBB5E0E0E9F5E0C0
:1007000080E0D81391C010928F0580918F05CC0F97
:10071000C82BC0938F0580918E05813009F088C069
:1007200010928E050E947B016B017C0180918F05E8
:100730008093BB008091B6059091B705A091B80554
:10074000B091B905892B8A2B8B2BA1F00E947B01DC
:100750000091B6051091B7052091B8053091B90503
:100760006C197D098E099F09061717072807390795
:1007700008F442C08091BC0083FDD8CF85EC809303
:10078000BC000E947B016B017C018091B40582302A
:1007900009F450C08091B2058F3F09F46FC0809179
:1007A000B205803209F46CC08091B205803309F43F
:1007B00069C084E026C08091B6059091B705A091EC
:1007C000B805B091B905892B8A2B8B2B09F484CFFE
:1007D0000E947B018090B6059090B705A090B80567
:1007E000B090B9056C197D098E099F098616970688
:1007F000A806B90608F070CF8091B5050E943303B2
:1008000085E01092BB051092DD051092BA05DF91CC
:10081000CF911F910F91FF90EF90DF90CF90BF90FD
:10082000AF909F908F9008959D9191938F5F69CF26
:1008300085EEA5CF8091B6059091B705A091B8053A
:10084000B091B905892B8A2B8B2B09F49ECF0E947E
:100850007B010091B6051091B7052091B805309144
:10086000B9056C197D098E099F0906171707280716
:10087000390708F08ACFC0CF81E0C3CF80E0C1CF75
:1008800082E0BFCF83E0BDCFCF93DF93EC018B81BC
:100890008823A1F0888191E09093BA058093DC05CC
:1008A0001092BB051092DD0581E00E94540391E097
:1008B000811190E0892FDF91CF9108951092AB04C0
:1008C0001092AA041092BB051092DD050E94150338
:1008D0008EED91E090939204809391048FED91E0DE
:1008E0009093900480938F0481E08B83CE010E94CB
:1008F0004404982F8111CECFDDCF0895E091AB0451
:100900008091AA04E81730F4F0E0E455FB4F8081B1
:1009100090E008958FEF9FEF08959091AB04809140
:10092000AA042FEF3FEF981748F4E92FF0E0E455C1
:10093000FB4F208130E09F5F9093AB04C901089585
:100940008091AA049091AB04891B990B0895CF92D2
:10095000DF92EF92FF920F931F93CF93DF937C016F
:10096000CB018A012091BA05222389F0EB016B01AA
:10097000C40ED51ECC15DD0569F06991D701ED9146
:10098000FC910190F081E02DC7010995F3CF642F10
:100990000E94EE02C801DF91CF911F910F91FF904D
:1009A000EF90DF90CF900895CF93DF931F92CDB754
:1009B000DEB769832091BA052223F9F02091DD0585
:1009C000203258F021E030E0FC013383228390E0B4
:1009D00080E00F90DF91CF9108958091BB05E82FC3
:1009E000F0E0E454FA4F998190838F5F8093BB05C8
:1009F0008093DD0581E090E0ECCF61E0CE010196CF
:100A00000E94EE02F7CF0895CF92DF92EF92FF920D
:100A10000F931F93CF93DF93EC0188858B7F88879B
:100A2000E881F9810190F081E02DCE010995182F20
:100A30008885869581701817B9F00E94D2016A8363
:100A40007B838C839D83888592E08927888788852E
:100A500082FB882780F9DF91CF911F910F91FF9042
:100A6000EF90DF90CF9008950E94D201CA80DB8082
:100A7000EC80FD80AB01BC014C195D096E097F095A
:100A80008E819F81B0E0A0E0481759076A077B0775
:100A9000F0F2888581701817D1F20E94D2016A8322
:100AA0007B838C839D83888591E0892784608887F8
:100AB0000E94D20109851A852B853C85601B710B2C
:100AC000820B930B6D877E878F87988B0E94D20154
:100AD00069877A878B879C87BACFCF93DF93EC01A6
:100AE0001886E881F9810190F081E02D099588232D
:100AF00019F08885836088870E94D2016A837B838E
:100B00008C839D83DF91CF910895862F642F0C9461
:100B10002D01FC0181890E94D60021E0892B09F476
:100B200020E0822F0895E7E0F5E021E084819581BF
:100B30008330910591F41582148210821182128201
:100B40001382379685E0EF33F80781F78FEF9FEF39
:100B500090936401809363010895049791F7108244
:100B60001182128213822683ECCF862F90916B051F
:100B7000992379F06CE00E943833E92FF0E0E650D9
:100B8000FE4F808187FD05C08093780181E08093CE
:100B90005D050895FB0140815181FC012081318177
:100BA000CA01821B930B08954F925F926F927F92BE
:100BB0008F929F92AF92BF92CF92DF92EF92FF926D
:100BC000CF938091850190918601029709F08DC0A5
:100BD000B0908405C1E08B2D8C2780937D050E9409
:100BE0007B016B017C01BB2009F477C08091E2039B
:100BF0009091E303A091E403B091E503A70196016E
:100C0000281B390B4A0B5B0BCA01B9010E94AC319E
:100C10004B015C0120917401309175014091760186
:100C2000509177010E94BB3220E030E044E353E46E
:100C30000E94043120E030E040E05FE30E94933006
:100C40000E947631DB0120EA30E00E9458332B010C
:100C50003C0124E130E040E050E00E946130211589
:100C6000310581E04807510508F04DC0C0934E059D
:100C70003093CE042093CD048091CD049091CE0486
:100C8000909387008093860080914E0580618093C9
:100C90008100C701B6010E94AC312B013C0120E06C
:100CA00030E040EC5FE3C501B4010E94BB329B0120
:100CB000AC01C301B2010E94933020E030E04AE76A
:100CC00054E40E9404310E947D316093800570934A
:100CD00081058093820590938305C092E203D092B0
:100CE000E303E092E403F092E503CF91FF90EF90ED
:100CF000DF90CF90BF90AF909F908F907F906F903C
:100D00005F904F9008952115310588E048075105FF
:100D100060F482E080934E05C301B20120EA30E026
:100D200040E050E00E946130A3CF2115310580E4FE
:100D30004807510550F483E080934E05C301B2018A
:100D400020E035E040E050E0EDCF211531054105D0
:100D500081E0580750F484E080934E05C301B2014E
:100D600020E034E140E050E0DDCF85E080934E05A7
:100D7000211531054105544038F4C301B20120E08A
:100D800030E540E050E0CECF8FEF9FEF9093CE0460
:100D90008093CD0471CFCF92DF92EF92FF92CF93E9
:100DA000DF938091850190918601892B29F08091B4
:100DB0008405882309F4A4C080917F058111A0C017
:100DC0008091DE039091DF03A091E003B091E103F5
:100DD0000196A11DB11D8093DE039093DF03A093C4
:100DE000E003B093E103C0900001D0900101409175
:100DF000DE035091DF036091E0037091E103C601CF
:100E0000D7FC019695958795092E000CAA0BBB0B74
:100E1000481759076A077B0750F080914F058823D0
:100E200031F010924F0560E081E00E94FF000D2C30
:100E3000000CEE08FF088091DE039091DF03A09183
:100E4000E003B091E1038C159D05AE05BF0508F4E4
:100E500057C0C1E0C0934F0561E081E00E94FF00F0
:100E6000C0937E056091DE037091DF038091E00303
:100E70009091E103A70196010E9461306093DE0327
:100E80007093DF038093E0039093E103209180014E
:100E90002E5F022E000C330BC9010896E8E0F0E04B
:100EA000BF010E944433EC01CD5BDA4FC9010796C4
:100EB000BF010E944433FC01ED5BFA4F88819081B1
:100EC000891B082E000C990B8C549F4F90930101A5
:100ED000809300012091FF04222391F020914A0485
:100EE0004CE350E0222311F044EC5FEF840F951F98
:100EF000909301018093000181E0282720934A0408
:100F0000DF91CF91FF90EF90DF90CF9008954F92B7
:100F10005F926F927F928F929F92AF92BF92CF9289
:100F2000DF92EF92FF92CF93DF93EC014A015B01D6
:100F30004C805D806E807F80A3019201CB01B40163
:100F40000E9492306B017C0120E030E0A9010E94F8
:100F5000B632181624F0F7FAF094F7F8F094A701D7
:100F60009601688579858A859B850E94FF3087FF79
:100F700017C08C829D82AE82BF826C817D818E8102
:100F80009F81DF91CF91FF90EF90DF90CF90BF9046
:100F9000AF909F908F907F906F905F904F9008954B
:100FA000C880D980EA80FB80A701960160E070E0EC
:100FB00080E89FE30E949230A30192010E94BB321D
:100FC0002B013C01A5019401C701B6010E94BB326F
:100FD0009B01AC01C301B2010E9493306C837D83FD
:100FE0008E839F83CACF90E080E00895DC011C9639
:100FF0008D919C91DC01ED91FC910484F585E02DAF
:101000000994CF92DF92EF92FF92CF93DF93FC018E
:10101000C485D5856B01770FEE08FF0860E079E0A5
:101020008DE390E0A70196010E94613021503109C3
:10103000410951095695479537952795E889F989CA
:1010400082E080832115F0E13F0798F0E889F98973
:10105000108260E874E88EE190E0A70196010E949A
:10106000613021503109410951095695479537950D
:101070002795EC85FD853083EE85FF852083188ECE
:10108000EC89FD8986E08083EA89FB898081806123
:101090008083EA89FB89808188608083EA89FB8973
:1010A000808180688083EA89FB8980818F7D80834D
:1010B000DF91CF91FF90EF90DF90CF900895DC010A
:1010C0001C968D919C91DC01ED91FC910284F3853D
:1010D000E02D0994DC011C968D919C91DC01ED9131
:1010E000FC910084F185E02D0994DC01ED91FD91E6
:1010F0008081ED91FD919081ED91FD916C916370F6
:101100008E2309F064609F2309F06860E2E9F8E04B
:10111000E60FF11D659565956D936D917D918D91AE
:101120009D91099423C01AC012C016C010C01EC0E1
:1011300009C014C013C006C019C009C00DC007C043
:101140000DC014C062507040804090400BC0615090
:1011500070408040904006C06E5F01C06F5F7F4F5F
:101160008F4F9F4F9E938E937E936E9308958091A1
:101170009304909194040C94750880919504909137
:1011800096040C947508089590E080E00895CF933C
:10119000DF93EC0160E08E810E94FF0061E08E81B0
:1011A0000E94FF0060E08E810E94FF008BE891E0CA
:1011B0000197F1F7DF91CF910895CF92DF92EF92EF
:1011C000FF920F931F93CF93DF936C017C0187E015
:1011D000E80EF11CD0E0C0E0062F10E0B8010C2EA4
:1011E00002C0759567950A94E2F76170F7018191E5
:1011F0007F010E94FF002196C430D10579F7C60116
:10120000DF91CF911F910F91FF90EF90DF90CF90E2
:101210000C94C708CF92DF92EF92FF920F931F9327
:10122000CF93DF93EC01F62E642F8C810E94FF0098
:101230008D818F3F19F060E00E94FF000F2D10E0BC
:101240008F8584FF25C06E0187E0C80ED11CF12C6C
:10125000E12CB8010E2C02C0759567950A94E2F74F
:101260006170F60181916F010E94FF00FFEFEF1A9C
:10127000FF0A88E0E816F10461F7CE01DF91CF9113
:101280001F910F91FF90EF90DF90CF900C94C708C3
:10129000B80184E0759567958A95E1F7CE010E94C3
:1012A000DD086F2DCE01DF91CF911F910F91FF903F
:1012B000EF90DF90CF900C94DD0840E0682F8BE03A
:1012C00096E00C940A0981E00E945D098BE39FE19E
:1012D0000197F1F70895CF93DF93823029F490912D
:1012E0001A06986090931A0680931E0610921F06A5
:1012F00080E48093200680E18093210680E580933E
:10130000220661E080910F060E942D018091100657
:101310008F3F19F061E00E942D0161E0809111067C
:101320000E942D01CBE0D6E09E012B5036408091EB
:101330001A0684FD0BC084E090E021962817390737
:1013400044F461E08E810E942D01EECF88E090E0B0
:10135000F4CF8BE39DE00197F1F760E080910F06F9
:101360000E94FF0060E0809111060E94FF008091C2
:1013700010068F3F19F060E00E94FF0080911A066E
:1013800084FD34C063E08BE096E00E94DD08CBE48E
:10139000D6E4CE010197F1F763E08BE096E00E947E
:1013A000DD082197F1F763E08BE096E00E94DD080D
:1013B00083E592E00197F1F762E08BE096E00E940E
:1013C000DD0880911A0680620E945D0984E08093A6
:1013D0001B068CE00E945D090E94630982E08093F5
:1013E0001C0686E0DF91CF910C945D0980620E941B
:1013F0005D098BE496E40197F1F780911A0680620B
:101400000E945D0983E592E00197F1F780911A0649
:1014100080620E945D09D5CF90911E06691710F079
:101420006FEF690FE62FF0E0E55FF94F9489890FC0
:1014300080680C945D0941E00E940A0981E090E017
:1014400008950F931F93CF93DF938B0128E0829F22
:10145000C001112480640E945D09E801085F1F4FEC
:1014600069918BE096E00E941B0AC017D107C1F773
:10147000DF91CF911F910F9108950F931F93CF93F9
:10148000DF938C01D0E0C0E0F801EC0FFD1F649108
:10149000662339F041E08BE096E00E940A0921962C
:1014A000F3CFCE01DF91CF911F910F9108958F92CD
:1014B0009F92AF92BF920F931F93CF93DF93CDB7BD
:1014C000DEB7A1970FB6F894DEBF0FBECDBF19A24D
:1014D000423008F44AE08E010F5D1F4F842E912C9C
:1014E000B12CA12CA50194010E946130E62FB90115
:1014F000CA01EA3044F5E05DD801EE938D01232B5B
:10150000242B252B79F790E080E0109769F0FD01FE
:1015100001900020E9F73197AF014A1B5B0BBD0139
:101520008BE096E00E94E101A1960FB6F894DEBF31
:101530000FBECDBFDF91CF911F910F91BF90AF90A4
:101540009F908F900895E95CD7CFCF92DF92EF9272
:10155000FF926B017C0141E06DE28BE096E00E941E
:101560000A0966277727CB016C197D098E099F0927
:101570004AE00E94570A0196FF90EF90DF90CF90CB
:101580000895BC01990F880B990B97FD0C94A50A3F
:101590004AE00C94570ACF9380917D0190917E018F
:1015A0000697A1F4C091830161E08C2F0E940C0A80
:1015B000EC2FCC0FFF0BE358FE4F8789082E000C51
:1015C000990B01960E94C10A10928301CF91089550
:1015D000009769F0FC0101900020E9F73197AF0115
:1015E000481B590BBC018BE096E00C94E10190E0A4
:1015F00080E008951F93CF93DF93C82F162F80911B
:101600008001DC2FD81B8C1784F5C093800180915A
:101610007D0190917E01069791F061E08DE00E943E
:101620000C0A8EE692E00E94E80A8C2FCC0F990BF0
:1016300001960E94C10A8BEE92E00E94E80AD15006
:1016400080915B05882321F060E083E00E94FF0029
:10165000C0E061E083E0CD1754F40E94FF0060E039
:1016600083E00E94FF00CF5FF4CFD85FCECF0E940F
:10167000FF000E947B01609357057093580580938B
:10168000590590935A0581E080935B05112339F049
:1016900060E080E1DF91CF911F910C94FF00DF911A
:1016A000CF911F910895CF92DF92EF92FF92CF9347
:1016B00020916F01309170012F3F3F4F09F07DC0A5
:1016C00020916D0130916E012F3F3F4F09F075C0A1
:1016D0006B017C0160E080E00E940C0A8091D304E1
:1016E000C0E0882329F08FE690E00E943D0AC3E025
:1016F0008AE690E00E943D0A8091850190918601E2
:10170000019709F120E030E040E85FE36091740167
:101710007091750180917601909177010E94FF3060
:10172000882389F088E690E00E943D0A80E792E0F5
:101730000E94E80AC75FCD3059F083E792E00E942B
:10174000E80ACF5FF8CF83E792E00E94E80AEECF85
:101750008091D30481111CC085E060E00E940C0AD6
:101760008091850190918601892B39F081E2C8161C
:1017700083E0D806E104F104BCF4F7FE0BC0C70116
:10178000B601CF91FF90EF90DF90CF900C94A50A17
:1017900088E0E3CF4AE0C701B601CF91FF90EF9018
:1017A000DF90CF900C94570A85E792E0CF91FF909D
:1017B000EF90DF90CF900C94E80ACF91FF90EF90DC
:1017C000DF90CF9008958F929F92AF92BF92CF9269
:1017D000DF92EF92FF92CF93DF93682F082E000CD9
:1017E000770BC0907401D0907501E0907601F09075
:1017F000770184300CF0F1C0C0918501D091860151
:101800006F5F7F4F072E000C880B990B0E94AE3143
:101810009B01AC0160E070E080E89FE30E9404312E
:101820006093100470931104809312049093130436
:10183000229751F4C1E0A70196010E94FF30811167
:1018400001C0C0E0C0931404809010049090110473
:10185000A0901204B0901304C1E0A7019601C50145
:10186000B4010E94FF30811101C0C0E0C0933F0568
:10187000A7019601C501B4010E94FF30882309F435
:101880000AC180911404811106C180927401909262
:101890007501A0927601B092770160910F01062E3A
:1018A000000C770B880B990B0E94AE31A5019401B7
:1018B0000E94BB320E947631AB0180914804909126
:1018C0004904BA010E944433909349048093480428
:1018D0009093420480934104609187017091880144
:1018E0008091890190918A010E94AE319B01AC01E7
:1018F00060EC71EE84E69CE40E940431A501940141
:101900000E94BB3220E030E044E353E40E94043103
:101910006B017C0120E030E0A9010E94B63220E09A
:1019200030E040E05FE387FD69C0C701B6010E9477
:1019300093300E947631A0EAB0E09B01AC010E9496
:1019400017306B017C0124E130E040E050E00E9460
:1019500061302115310581E04807510508F053C079
:1019600081E080934E053093CE042093CD04809186
:10197000CD049091CE04909387008093860080914F
:101980004E05806180938100809185019091860150
:10199000892B09F080C06091870170918801809146
:1019A000890190918A010E94AE3120917401309199
:1019B000750140917601509177010E9404310E9497
:1019C0007631DF91CF91FF90EF90DF90CF90BF9075
:1019D000AF909F908F900C94530B63507109072E1A
:1019E000000C880B990B0E94AE3160931004709329
:1019F0001104809312049093130426CFC701B601FB
:101A00000E94923096CF2115310588E04807510594
:101A100060F482E080934E05C701B60120EA30E011
:101A200040E050E00E9461309ECF2115310580E4F6
:101A30004807510550F483E080934E05C701B60175
:101A400020E035E040E050E0EDCF211531054105C3
:101A500081E0580750F484E080934E05C701B60139
:101A600020E034E140E050E0DDCF85E080934E059A
:101A7000211531054105544038F4C701B60120E075
:101A800030E540E050E0CECF8FEF9FEF9093CE0453
:101A90008093CD046CCFDF91CF91FF90EF90DF90DA
:101AA000CF90BF90AF909F908F9008950F931F930A
:101AB000CF9360E080E00E940C0A05E611E0C0E0F0
:101AC00082E792E00E94E80AF80181918F01082ED6
:101AD000000C990B0E94C10ACF5FC83021F4CF914E
:101AE0001F910F910895C43059F761E080E00E9482
:101AF0000C0AE6CFEF92FF921F93CF93DF9360E043
:101B000080E00E940C0A83E4E82E85E0F82E10E0C5
:101B1000D0E0F701C1917F01C73F54F58C2FCC0F66
:101B2000990B0E94C10AD11107C0D1E0F70131978A
:101B30008081811101C0D0E01F5F183091F4DD2356
:101B400041F08091850190918601D1E0892B09F4C3
:101B5000D0E0D0938405DF91CF911F91FF90EF905B
:101B600008951430B1F661E080E00E940C0AD1CFF4
:101B7000C7FF05C083E792E00E94E80ACFCF88E75D
:101B800092E0CA30CCF787E792E0C111F5CF8AE73F
:101B900092E00E94E80AC7CFCF9390917F019817F7
:101BA000C1F0C82F80937F0160E08EE00E940C0A94
:101BB00080917D0190917E01069729F48EE792E055
:101BC000CF910C94E80A8C2FCC0F990BCF910C94E9
:101BD000C10ACF910895EF92FF920F931F93CF9375
:101BE000DF937C01042FC22F842F0E940C0AC701AF
:101BF0000E94E80AF70101900020E9F73197EE19F9
:101C0000FF09D0E00E0F1F2F111D0C171D0734F414
:101C100083E792E00E94E80A2197F7CFDF91CF9106
:101C20001F910F91FF90EF9008958F929F92AF9226
:101C3000BF92CF92DF92EF92FF920F931F93CF93B9
:101C4000DF936B018A01E901219720E140E060E028
:101C50000E94EB0D99E1E92E9CEFF92EA0904C0526
:101C6000B0904D05F5018385823008F047C0F894A7
:101C7000C5010E947508F50187809084A184B28413
:101C800078946091710170917201C4010E94443393
:101C9000892B59F4C4018E199F091816190684F16D
:101CA0008FEF9FEF8E149F0469F58091400590910E
:101CB00041050E940405E0914005F09141058085B1
:101CC00080FD1AC082FF18C0E0914C05F0914D05CF
:101CD000F89417821086118612867894CE01DF91CF
:101CE000CF911F910F91FF90EF90DF90CF90BF9019
:101CF000AF909F908F9008957401B0CFF894BBCFB0
:101D000081E090E0C80FD91FD7FF0FC0C00FD11FCF
:101D1000FE01EE0FFF1FEC0DFD1D20E140E061E034
:101D2000808191810E94EB0DC0CFC017D10784F351
:101D3000C01BD10BEDCFCF93DF93EB012DE040E043
:101D400060E00E94EB0DCF3F8FEFD80741F01CF011
:101D5000C530D10534F0CE01DF91CF910895D0E0A8
:101D6000C0E0FE01EE0FFF1FE051FE4F2DE040E00E
:101D700061E0808191810E94EB0DEDCFCF93809146
:101D8000A00481113CC080916B05811143C0E0919A
:101D90007D01EC30A9F561E00E940C0A87E892E031
:101DA0000E94E80A8091FF04811126C084E892E035
:101DB0002DE04AE061E00E94EB0D80917D01909161
:101DC0007E01069709F046C061E080E00E940C0A9F
:101DD000C0E040918401C417FCF4EC2F0C2E000CE1
:101DE000FF0BE358FE4F8789082E000C990B0196D4
:101DF0000E94C10ACF5FEDCF80E892E0D9CFE7E043
:101E0000EE0FFF0BE25FFD4F2DE040E060E08081D0
:101E10009181D1CFE8E0F4CF403134F420E161E0AA
:101E200084E792E00E94EB0D809184018A3084F077
:101E30008CE060E00E940C0A8EE692E00E94E80AC4
:101E400080918401082E000C990B0E94C10A16C0D3
:101E50008DE0EFCF60E08DE00E940C0A8EE692E00C
:101E60000E94E80A80916B05882369F08091A104A3
:101E7000181644F38EE792E00E94E80A8BEE92E097
:101E8000CF910C94E80A80917F01DCCF1092650518
:101E90000E94BE0E61E080E00E940C0A83E790E0A1
:101EA0000C943D0A4F925F926F927F928F929F9215
:101EB000AF92BF92CF92DF92EF92FF92CF93809139
:101EC000850190918601019709F0EEC0B0908405DC
:101ED000C1E08B2D8C2780937C050E947B016B01D8
:101EE0007C01BB2009F46DC08091440490914504AD
:101EF000A0914604B0914704A7019601281B390B15
:101F00004A0B5B0BCA01B9010E94AC314B015C0169
:101F100020E030E044E353E40E94043120E030E06C
:101F200040E05FE30E9493300E947631DB0120EABB
:101F300030E00E9458332B013C0124E130E040E0C6
:101F400050E00E9461302115310581E048075105BC
:101F500008F062C0C0934E053093CE042093CD04A8
:101F60008091CD049091CE04909387008093860059
:101F700080914E05806180938100C701B6010E9467
:101F8000AC312B013C0120E030E040EC5FE3C501C7
:101F9000B4010E94BB329B01AC01C301B2010E949B
:101FA000933020E030E04AE754E40E9404310E947C
:101FB0007D316093800570938105809382059093B5
:101FC0008305C0924404D0924504E0924604F09206
:101FD000470480917C05882309F466C00E94D201E1
:101FE0006093660570936705809368059093690513
:101FF00080916505882309F457C0CF91FF90EF9039
:10200000DF90CF90BF90AF909F908F907F906F9018
:102010005F904F900C94460F2115310588E04807DA
:10202000510560F482E080934E05C301B20120EABD
:1020300030E040E050E00E9461308ECF2115310544
:1020400080E44807510550F483E080934E05C301B6
:10205000B20120E035E040E050E0EDCF2115310540
:10206000410581E0580750F484E080934E05C30198
:10207000B20120E034E140E050E0DDCF85E0809324
:102080004E05211531054105544038F4C301B20114
:1020900020E030E540E050E0CECF8FEF9FEF90930F
:1020A000CE048093CD045CCFCF91FF90EF90DF9072
:1020B000CF90BF90AF909F908F907F906F905F90E8
:1020C0004F900895CF9380917D0190917E01C091B2
:1020D0008C018430910599F058F4E0917F01CFEFA5
:1020E000CE0F8130910559F00297D9F0C0E007C0BA
:1020F00085309105D1F0C09194010697B9F71092FF
:1021000082011092830160E08C2F0E94FA0AEC2F6A
:10211000CC0FFF0BEB59FE4F808180939F04CF9132
:10212000089581E080938101E1CF0E94BE2F892F25
:10213000990F990B60917F01062E000C770B0E947E
:102140004433C82FDCCF809185019091860101979F
:1021500021F480917C0581110AC0809185019091C4
:1021600086010297C1F480917D058823A1F08091BA
:102170005E058823A9F010925E050E94CB0A0E949A
:10218000621010925D0560914F0581E068276093B1
:102190004F050E94FF0010927C0510927D05089566
:1021A00081E080935D05EFCFCF93DF938091FF04B3
:1021B000882399F080EF90E09093010180930001D3
:1021C00081E080934A0480918B01882369F181E04A
:1021D00080935E05DF91CF910895E09180010E2EEE
:1021E000000CFF0BCF010296C8E0D0E0BE010E94B8
:1021F0004433DC01AD5BBA4F2C91022E000C330B43
:102200002C543F4FCF010196BE010E944433FC0184
:10221000ED5BFA4F8081281B310987FD33953093A0
:10222000010120930001CFCF0E946210DF91CF9176
:102230000C94CB0ACF93DF93C82FD62F80938B01BA
:1022400084EB90E090930101809300016C2F8DE06E
:102250000E94FF0080915C0561E0811101C06C2744
:1022600080E10E94FF00DD2321F0DF91CF910C94EB
:10227000D4108091FF04882341F080EF90E0909388
:1022800001018093000110924A04DF91CF910895DB
:1022900010927E058091850190918601892B21F015
:1022A00080918405882389F080915E05882331F030
:1022B00010925E050E94CB0A0C94621080918B01F3
:1022C000882319F081E080935D0508950E948A3487
:1022D00085ED8093BC008091B6059091B705A091E3
:1022E000B805B091B9050796A11DB11D23E0B695BB
:1022F000A795979587952A95D1F72091BC0024FD45
:1023000003C01092B40508954091B6055091B705E9
:102310006091B8057091B905452B462B472B69F3A1
:102320000097A105B10541F02AE22A95F1F700C016
:102330000197A109B109E1CF8091B5050C94330350
:10234000FF920F931F93CF93DF938C01EB01F880E3
:102350000E94CE2FF81621F06F2DC8010E94D62FB3
:10236000CE01DF91CF911F910F91FF900895FF92C1
:102370000F931F93CF93DF93EC018B01FB01F08050
:102380000E94CE2FF81621F06F2DCE010E94D62F7D
:10239000F801F1802196CE010E94CE2FF81621F08F
:1023A0006F2DCE010E94D62FC801DF91CF911F91D2
:1023B0000F91FF9008950F931F93CF93DF938C019C
:1023C000EB010E94CE2F8883C80101960E94CE2F78
:1023D0008983CE01DF91CF911F910F910895FC0168
:1023E0009AE2A6EEB3E001900D929A95E1F72AECFD
:1023F00035E042E050E065E170E086EE93E00E9457
:10240000052E8091FA039091FB03089510924404E5
:1024100010924504109246041092470410927B05D6
:1024200010927A051092790110927A0110927B0134
:1024300010927C011092400410923F04882339F0DE
:10244000E5E1F4E08AE2DF011D928A95E9F708955B
:10245000EF92FF920F931F93CF93DF9380914205EA
:10246000893081F420E140E061E082E992E00E945D
:10247000EB0D10928001DF91CF911F910F91FF9092
:10248000EF9008958D3009F097C080916F01909181
:1024900070018230910509F465C05CF58F3F9807A3
:1024A000A9F1892B09F445C080916F0190917001C9
:1024B000019609F04EC00E94BE0E2DE040E061E0A2
:1024C0008DE992E00E94EB0DE3E4F5E025E0EB34CA
:1024D000F20709F46BC081918823C1F381E08093F6
:1024E000CC042091850130918601232B09F061C035
:1024F0005FC08330910509F44DC00497A9F68FEFB2
:102500009FEF9093700180936F01CECF1092700176
:1025100010926F012DE040E060E08DE992E00E94B2
:10252000EB0D2DE040E061E089EA92E00E94EB0DC6
:10253000BBCF1092430510924405109245051092AE
:1025400046051092470510924805109249051092D1
:102550004A0581E090E09093700180936F010E94A2
:102560007A0DB2CF03E415E097E9E92E94E0F92E55
:10257000CEE1D0E0D8018C91F70181937F01B801C1
:10258000CE010E94A0110F5F1F4F2296CE32D105BF
:1025900089F78ACFE7E9F4E0A3E4B5E08FE994E0B6
:1025A00021912D938E179F07D9F7D3CF1092CC048A
:1025B00080E0809384055FCF8B3009F086C08091E6
:1025C0006D0190916E018230910509F45BC0DCF4DD
:1025D0008F3F980729F1892BB1F180916D0190917E
:1025E0006E01019609F040C00E94BE0E2DE040E051
:1025F00061E08FEA92E0DF91CF911F910F91FF9000
:10260000EF900C94EB0D8330910509F453C00497BF
:1026100021F78FEF9FEF90936E0180936D01DDCFD7
:1026200010926E0110926D012DE040E060E08FEAA3
:1026300092E00E94EB0D2DE040E061E089EA92E03B
:102640000E94EB0DCACF81E0809365018093660103
:1026500080936701809368018093690180936A0188
:1026600080936B0180936C0181E090E090936E0108
:1026700080936D01DF91CF911F910F91FF90EF90AB
:102680000C94560D05E611E086E0E82E81E0F82E68
:10269000CAE0D0E0F8018081D7018D937D01B801B7
:1026A000CE010E94A0110F5F1F4F2296CA31D105A3
:1026B00089F793CFE6E0F1E0A5E6B1E081918D9353
:1026C00021E0EE30F207D1F7CFCF10926B05C09129
:1026D000A004CC23A9F01092A0040E94BE0E809109
:1026E000A004882309F485C020E140E061E084E78C
:1026F00092E00E94EB0D1092830110928401BBCEF8
:10270000873064F5809100059091010590937E01DA
:1027100080937D018230910521F481E080938101D5
:10272000DCCF0497D1F60DE711E0C8E0D0E00E94BD
:10273000BE2FBE010E944433F8012689FC01E358F4
:10274000FE4F8785D80156968C9327872197015095
:102750001109209761F710928201BFCF91E0873075
:1027600009F090E09093A00491E0883009F090E0A7
:1027700090936B058C3089F58091FF0491E0892757
:102780008093FF0461E080E00E940C0A87E892E0F9
:102790000E94E80A8091FF04882341F180E892E0DA
:1027A0002DE04AE061E00E94EB0D8091850190915F
:1027B0008601892B81F0C091CC04C1110CC0C0915D
:1027C000FF04CC2341F08091850190918601C1E006
:1027D000019709F0C0E0C0938405109202051092A1
:1027E0000305109204051092050577CF84E892E066
:1027F000D7CF80916B05882331F020E140E061E084
:1028000084E792E0F8CE809142058A3009F033CE19
:102810008091850190918601892B31F020E140E083
:1028200061E089EB92E0E7CE8091060581110DC051
:1028300081E08093D304809306050E94061220E174
:1028400040E061E088EC92E0D6CE1092060520E1EF
:1028500040E061E083ED92E00E94EB0D6091790130
:1028600070917A0180917B0190917C010E94763178
:1028700060938701709388018093890190938A0106
:102880000E94AE3120917401309175014091760122
:10289000509177010E9404310E947631DF91CF91EF
:1028A0001F910F91FF90EF900C94530B8091850135
:1028B00090918601029709F046C0842F90E024E0B1
:1028C000959587952A95E1F78770613171F06231AE
:1028D00079F16031C1F520917D0130917E01263082
:1028E000310589F18F5F0C94CC0D873061F1482F51
:1028F00050E020914205022E000C330B4217530783
:1029000011F180934205509301054093000561E069
:1029100080E00E940C0A83E790E00E943D0A8091CB
:102920003F05882319F010923F0508950C94281252
:10293000873049F0843018F083500C94E30B47E063
:10294000481B842FFACF08954F925F926F927F9227
:102950008F929F92AF92BF92CF92DF92EF92FF92AF
:10296000CF93DF9300D000D01F92CDB7DEB7809118
:10297000850190918601029709F01FC3442321F13C
:102980008091850190918601029709F016C381E03C
:102990008093430480910E0181110FC360E00F907A
:1029A0000F900F900F900F90DF91CF91FF90EF90CD
:1029B000DF90CF90BF90AF909F908F907F906F905F
:1029C0005F904F900C941A11662379F180918501E4
:1029D00090918601029709F0F0C21092430480E0C2
:1029E0000E9406128FEF9FEF909349048093480452
:1029F000909342048093410461E081E00E941A11A7
:102A00000F900F900F900F900F90DF91CF91FF904C
:102A1000EF90DF90CF90BF90AF909F908F907F907E
:102A20006F905F904F900C94D4052223B9F0809161
:102A3000850190918601029709F0BFC2109243046C
:102A400080910E018111B9C20E9406128FEF9FEF93
:102A5000909349048093480460E0CFCF809148046C
:102A60009091490401969093490480934804809181
:102A70004104909142040196909342048093410452
:102A8000209140042F5F2D83209340040E947B01FE
:102A900069837A838B839C8380914404909145045D
:102AA000A0914604B0914704892B8A2B8B2B09F403
:102AB000B4C0409044045090450460904604709027
:102AC000470460910F01062E000C770B880B990BC1
:102AD0000E94AE31209174013091750140917601D0
:102AE000509177010E94BB329B01AC0160E070E61F
:102AF0008AE697E40E9404316B017C0169817A8146
:102B00008B819C810E94AC314B015C01C301B201FD
:102B10000E94AC319B01AC01C501B4010E9492300E
:102B20009B01AC01C701B6010E94043120E030E0F6
:102B30004AE754E40E94BB326B017C0120E030E0A4
:102B4000A9010E94B63220E030E040E05FE387FD5B
:102B500017C1C701B6010E9493300E9476314090A0
:102B6000790150907A0160907B0170907C01809196
:102B70003F04082E000C990BFC01EE0FFF1FEB5ECB
:102B8000FB4F71836083019665E170E00E944433DE
:102B900080933F048D8185318CF085E194E00E9423
:102BA000EF11BC0190E080E00E94AC3160937901AC
:102BB00070937A0180937B0190937C01A301920131
:102BC0006091790170917A0180917B0190917C01F3
:102BD0000E9492304B015C0120E030E0A9010E948C
:102BE000B632181624F0B7FAB094B7F8B094A3012F
:102BF0009201C501B4010E94043120E030E040E8B8
:102C00005EE30E94B632181644F4C0927901D09265
:102C10007A01E0927B01F0927C0189819A81AB81FB
:102C2000BC818093440490934504A0934604B093E0
:102C30004704D0900F016D2D0D2C000C770B880BE5
:102C4000990B0E94AE314B015C01209174013091CF
:102C5000750140917601509177010E94BB322B01A2
:102C60003C0120E030E0A9010E94B63220E030E0D3
:102C700040E05FE387FD89C0C301B2010E94933049
:102C80000E9476317B018091FF04882301F1C70106
:102C900063E070E00E944433072E000C880B990B10
:102CA0000E94AE3120914A04222309F476C020E02C
:102CB00030E040E05FE3AEEFEA16AFEFFA060CF467
:102CC00069C00E9493300E947631E60EF71E809113
:102CD0004804909149048E159F0509F06EC18091BA
:102CE0004A0491E0892780934A0410924904109283
:102CF000480480911404882309F4E7C06D2DDD0C8D
:102D0000770B80914104909142040E944433892BB7
:102D100009F0DBC010921404109242041092410496
:102D2000C0901004D0901104E0901204F0901304AD
:102D3000C0927401D0927501E0927601F092770111
:102D400080918501909186010297D1F18091D30401
:102D5000811136C08091850190918601892B09F0FF
:102D600056C060918701709188018091890190918E
:102D70008A010E94AE31A70196010E94043143C02E
:102D8000C701B6010E949230E8CEC301B2010E9491
:102D9000923076CF0E94923096CF20E030E040E033
:102DA0005FE3BEEFEB16BFEFFB063CF00E949330F3
:102DB0000E947631E61AF70A8ACF0E949230F8CF45
:102DC0002091790130917A0140917B0150917C01F1
:102DD000C501B4010E94BB3220E030E040EC51E478
:102DE0000E9404316B017C0120E030E0A9010E94C7
:102DF000B63220E030E040E05FE387FDF2C0C7017B
:102E0000B6010E9493300E9476310E94530B60916C
:102E10008701709188018091890190918A010E94B7
:102E2000AE319B01AC0160EC71EE84E69CE40E9443
:102E300004312091740130917501409176015091D7
:102E400077010E94BB3220E030E044E353E40E946B
:102E500004316B017C0120E030E0A9010E94B63210
:102E600020E030E040E05FE387FDC0C0C701B6016D
:102E70000E9493300E947631A0EAB0E09B01AC0141
:102E80000E9417306B017C0124E130E040E050E00B
:102E90000E9461302115310581E04807510508F095
:102EA000AAC081E080934E053093CE042093CD04D8
:102EB0008091CD049091CE049093870080938600FA
:102EC00080914E05806180938100809144049091AF
:102ED0004504A0914604B0914704892B8A2B8B2B83
:102EE00009F45DC0C0907901D0907A01E0907B0137
:102EF000F0907C01B701A6018BEF95E00E94870757
:102F000020E030E0A9010E94B632B701A60187FD9A
:102F1000BAC08BEF95E00E94870720E030E040E0E8
:102F20005FE30E9493300E9476316B017C018091B7
:102F30007A0590917B05092E000CAA0BBB0B8C1512
:102F40009D05AE05BF0559F1A0910F010A2E000C99
:102F5000BB0BA70196010E9422304B015C0128E1C6
:102F600030E040E050E00E94F82FCA01B9010E9411
:102F7000AE3120E030E040E05FE3A9EE8A16AFEF2B
:102F80009A06AA06BA060CF489C00E9493300E94E1
:102F900076310E94530BD0927B05C0927A058091C6
:102FA0008B01882351F080910E01882309F428CDEC
:102FB00080914304882309F423CD0F900F900F9044
:102FC0000F900F90DF91CF91FF90EF90DF90CF9017
:102FD000BF90AF909F908F907F906F905F904F9039
:102FE0000895C701B6010E9492300DCFC701B60106
:102FF0000E9492303FCF2115310598E049075105D5
:1030000060F482E080934E05C701B60120EA30E00B
:1030100040E050E00E94613047CF21153105A0E427
:103020004A07510550F483E080934E05C701B6016D
:1030300020E035E040E050E0EDCF211531054105BD
:10304000B1E05B0750F484E080934E05C701B60100
:1030500020E034E140E050E0DDCF85E080934E0594
:10306000211531054105544038F4C701B60120E06F
:1030700030E540E050E0CECF8FEF9FEF9093CE044D
:103080008093CD0415CF8BEF95E00E94870720E059
:1030900030E040E05FE30E94923045CF0E949230E2
:1030A00076CF1F920F920FB60F9211242F933F935A
:1030B0008F939F93AF93BF938091860590918705DF
:1030C000A0918805B09189053091850523E0230FF3
:1030D0002D3758F50196A11DB11D209385058093CC
:1030E000860590938705A0938805B0938905809104
:1030F0008A0590918B05A0918C05B0918D05019664
:10310000A11DB11D80938A0590938B05A0938C051A
:10311000B0938D05BF91AF919F918F913F912F916A
:103120000F900FBE0F901F90189526E8230F029660
:10313000A11DB11DD2CF1F920F920FB60F92112475
:103140002F933F934F935F936F937F938F939F93AF
:10315000AF93BF93EF93FF93E0910401F0910501CA
:103160000995FF91EF91BF91AF919F918F917F91C1
:103170006F915F914F913F912F910F900FBE0F90E4
:103180001F9018951F920F920FB60F9211242F9334
:103190003F934F935F936F937F938F939F93AF93DF
:1031A000BF93EF93FF93E0910201F0910301099522
:1031B000FF91EF91BF91AF919F918F917F916F910F
:1031C0005F914F913F912F910F900FBE0F901F90E5
:1031D00018951F920F920FB60F9211242F933F93C1
:1031E0004F935F936F937F938F939F93AF93BF930F
:1031F000EF93FF9388E496E00E945F02FF91EF91C6
:10320000BF91AF919F918F917F916F915F914F91FE
:103210003F912F910F900FBE0F901F9018951F9206
:103220000F920FB60F9211242F938F939F93EF93CA
:10323000FF93E0915806F09159068081E0915E0677
:10324000F0915F0682FD1BC09081809161068F5FC7
:103250008F7320916206821741F0E0916106F0E0E1
:10326000E85BF94F958F80936106FF91EF919F91F5
:103270008F912F910F900FBE0F901F901895808106
:10328000F4CF1F920F920FB60F9211242F933F93FA
:103290004F935F936F937F938F939F93AF93BF935E
:1032A000EF93FF938091B900887F803609F44AC07C
:1032B000F0F5883209F4A7C018F5803109F49BC0F5
:1032C000B8F4882309F4F9C0883009F494C0FF9158
:1032D000EF91BF91AF919F918F917F916F915F918E
:1032E0004F913F912F910F900FBE0F901F90189507
:1032F000883109F488C0803251F78093B20514C038
:10330000803409F49DC040F48033B9F38833F9F672
:103310008093B20585ECB0C0803509F485C088354E
:1033200009F496C0883499F60E946811D0CF883984
:1033300009F48CC038F5883729F050F4883611F03C
:10334000803729F683E08093B40510928E0457C02D
:10335000883809F47BC0803919F0803809F0B7CF7C
:1033600080918E04803208F071C0E0918E0481E07B
:103370008E0F80938E048091BB00F0E0E259FB4FEA
:1033800080833DC0803B39F0E0F4803A09F479C095
:10339000883A09F09CCF84E08093B40510926D04C4
:1033A00010926C04E0919104F0919204099580913F
:1033B0006C0481110FC081E080936C0410924C0466
:1033C00009C0803C09F4A6CF883C09F4A3CF883B10
:1033D00009F07DCFE0916D0481E08E0F80936D0444
:1033E000F0E0E45BFB4F80818093BB0090916D0423
:1033F00080916C0429C080918F058093BB0085EC7F
:103400008093BC0064CF9091B1058091B00598176E
:1034100058F5E091B10581E08E0F8093B105F0E0A1
:10342000E057FA4F8081E9CFE091B10581E08E0F3E
:103430008093B1058091BB00F0E0E057FA4F8083A4
:103440009091B1058091B0059817C8F285E8D8CF62
:10345000E091B10581E08E0F8093B1058091BB00B2
:10346000F0E0E057FA4F80838091B30581115CCF83
:1034700081E080938E0584EA8093BC001092B405AD
:1034800026CF85EC8093BC001092B40580918E0409
:10349000803230F4E0918E04F0E0E259FB4F10826C
:1034A00060918E0470E0E0918F04F09190048EE6BC
:1034B00094E0099510928E040ACF1092B20534CF91
:1034C0001F920F920FB60F9211242F933F934F9399
:1034D0005F936F937F938F939F93AF93BF93EF937C
:1034E000FF93E0911001F09111010995FF91EF9187
:1034F000BF91AF919F918F917F916F915F914F910C
:103500003F912F910F900FBE0F901F901895109222
:103510004B0610924A0688EE93E0A0E0B0E080935C
:103520004C0690934D06A0934E06B0934F062EE2A4
:1035300032E0309349062093480625EC30E0309382
:1035400055062093540624EC30E030935706209320
:10355000560620EC30E0309359062093580621ECB3
:1035600030E030935B0620935A0622EC30E0309333
:103570005D0620935C0626EC30E030935F062093D6
:103580005E06109261061092620610926306109217
:1035900064061092E1051092E0058093E205909395
:1035A000E305A093E405B093E50520E432E0309311
:1035B000DF052093DE051092EA051092EB051092CC
:1035C000E8061092E7068093E9069093EA06A09336
:1035D000EB06B093EC068EE592E09093E6068093BE
:1035E000E50688E496E09093F2068093F10685EE76
:1035F00096E090932406809323061092260610925C
:103600002506109228061092270681E090E09093FC
:10361000300680932F0690933206809331061092E5
:103620000E0610920D0682E592E090930C068093B0
:103630000B0688E080930F068FEF8093100689E0D9
:103640008093110684E08093120685E08093130630
:1036500086E08093140687E0809315061092160684
:1036600010921706109218061092190610921A0658
:1036700081E00E946B090E94D2016093070670935B
:1036800008068093090690930A060E94D2018AE9EF
:1036900099E9A9E9BEE38093FB059093FC05A0930B
:1036A000FD05B093FE0580E090E0A0EFB2E48093CA
:1036B000FF0590930006A0930106B093020680E0F8
:1036C00090E0A0E4B0E48093030690930406A093F6
:1036D0000506B09306068091FA05811125C080E0A9
:1036E00090E0A0E0B0E44AE959E969E97EE340935B
:1036F000EE055093EF056093F0057093F10540E0FF
:1037000050E060EF72E44093F2055093F30560934C
:10371000F4057093F5058093F6059093F705A09353
:10372000F805B093F905089580E090E0A0E4B0E4D6
:10373000DACFCF93DF93CDB7DEB7CA54D1090FB636
:10374000F894DEBF0FBECDBF789484B5826084BD8F
:1037500084B5816084BD85B5826085BD85B5816095
:1037600085BD80916E00816080936E001092810013
:1037700080918100826080938100809181008160CE
:10378000809381008091800081608093800080918F
:10379000B10084608093B1008091B000816080931B
:1037A000B00080917A00846080937A0080917A00E2
:1037B000826080937A0080917A00816080937A00A1
:1037C00080917A00806880937A001092C10082E034
:1037D0000E946B0988E00E945D0986E00E945D09F5
:1037E00087E10E945D0981E00E945D0982E00E94FC
:1037F0005D098CE00E945D090E94630982E00E94DD
:103800005D098BE39FE10197F1F78CED92E00E9457
:10381000E80A6AE471E080E00E94210A62E471E053
:1038200081E00E94210A6AE371E082E00E94210A9D
:1038300062E371E083E00E94210A6AE271E084E0C1
:103840000E94210A62E271E085E00E94210A6AE199
:1038500071E086E00E94210A62E171E087E00E9447
:10386000210A8091EC059091ED050E94013486E0DB
:1038700090E00E9465338C0180E2D8018C938EED3C
:1038800095E012969C938E93119713961C92139722
:1038900080E290E015969C938E9314971093ED051B
:1038A0000093EC051092AB041092AA041092BB0591
:1038B0001092DD050E9415038EED91E09093920425
:1038C000809391048FED91E09093900480938F0406
:1038D00081E0F8018383C8010E94440410E000E005
:1038E000EE24E394F12CDD24D3948091EB05970131
:1038F000002E01C0220F0A94EAF7822B8093EB0579
:10390000E091EC05F091ED0584819581892BD9F04A
:10391000818192812081D092BA052093DC0510929A
:10392000BB051092DD05DC01ED91FC910280F38175
:10393000E02D41E050E06BEE75E00995019719F438
:1039400081E00E9454030F5F1F4F0830110569F694
:1039500062E08EE00E942D0162E081E10E942D0173
:1039600062E08AE00E942D0162E08BE00E942D015E
:103970008CE090E00E9465338C0162E08AE00E9456
:103980002D0162E08BE00E942D01E2EDF0E0E49178
:10399000F0E0EE0FFF1FE254FF4FA591B491F80144
:1039A000B183A083E6EEF0E08491F8018483E3ED37
:1039B000F0E0E491F0E0EE0FFF1FE254FF4F25919D
:1039C0003491F80133832283E7EEF0E06491F8014B
:1039D000658317821086118612864BE35FE1FA0138
:1039E0003197F1F79C91892391E009F490E0D90196
:1039F0008C91E62FE82309F09260F80196831386F4
:103A000010934D0500934C0562E08CE00E942D015F
:103A100082E190E00E946533FC01128213821482DD
:103A20001582AAE0CA2ED12CD782C6821086BAE0AF
:103A3000EB2EB2E0FB2EF182E08290934105809361
:103A400040058CE0818BCF010E946D05E09140051F
:103A5000F091410502E310E01783068362E08FE0F6
:103A60000E942D0182E190E00E946533FC011282E8
:103A7000138214821582D782C6821086F182E08278
:103A800090935605809355058FE0818BCF010E945E
:103A90006D05E0915505F09156051783068361E0A9
:103AA0008DE00E942D0160918B018DE00E94FF004E
:103AB00061E083E00E942D0160E083E00E94FF004E
:103AC00061E080E10E942D0161E080E10E94FF0041
:103AD00062E082E00E942D0182E59FE09093030165
:103AE00080930201809169008C7F826080936900DD
:103AF000E89A60E084E10E942D0180E180938100DA
:103B00001092800083E080934E0584E294EF9093BE
:103B1000CE048093CD04909387008093860083E148
:103B2000809381008BEC96E09093110180931001BB
:103B300081E080936F0085EB95E09093370680934A
:103B40003606109239061092380684EA94E1909372
:103B500041068093400686E594E190933B0680936E
:103B60003A060091A104002E000C110B809123064F
:103B700090912406DC01ED91FC910684F785E02DFF
:103B800062E17AE7099510922606109225061093B5
:103B9000300600932F068091C100877F8093C1007B
:103BA00061E081E00E942D0110924F0560E081E00C
:103BB0000E94FF0086E0EEEAF1E0DE0195960190BA
:103BC0000D928A95E1F7BE01655C7F4F90E080E041
:103BD0000E94DB112BAD3CAD2230310538F481E081
:103BE000121613060CF080E080935C05BE01675C42
:103BF0007F4F82E090E00E94DB1189AD9AAD9C017D
:103C0000215031092730310510F48093A104BE0101
:103C1000695C7F4F84E090E00E94DB112FA938ADF2
:103C20002230310538F481E0121613060CF080E0E2
:103C30008093FA05BE016F5C7F4F86E090E00E94A2
:103C4000DB1189A99AA963E070E00E94E42F9AAB86
:103C500089AB880F991FFE0131961F01E80FF91FEC
:103C600084A180930F01BE016B5C7F4F88E090E0E0
:103C70000E94DB112DA93EA92115310521F08FA944
:103C800098AD019739F481E0121613060CF080E02C
:103C900080930E01BE016D5C7F4F8AE090E00E9430
:103CA000DB118BA99CA98230910519F08430910514
:103CB00021F490937201809371018091400590915D
:103CC00041050E940405E0914005F0914105808581
:103CD00080FDCAC08091B4019091B501A091B60158
:103CE000B091B7018BA79CA7ADA7BEA720915C059B
:103CF00030E042E050E0BE01655D7F4F8DEE92E026
:103D00000E94150E21E0019709F020E020935C0548
:103D100030E03A832983B10190E080E00E94B7113E
:103D200064EF71E080E090E00E94A0012091FA052C
:103D300030E042E050E0BE01655D7F4F8CEF92E0E5
:103D40000E94150E21E0019709F020E02093FA056A
:103D500030E03A832983B10184E090E00E94B711FA
:103D600064EF71E080E090E00E94A00186E0E8EB63
:103D7000F1E0D10101900D928A95E1F729A93AA9C4
:103D800043E050E0B10189E093E00E94150EFC0190
:103D9000EE0FFF1FE20DF31D24A120930F019E8B58
:103DA0008D8BBE016B5E7F4F86E090E00E94B71165
:103DB00064EF71E080E090E00E94A00120910E018C
:103DC00030E042E050E0BE01655D7F4F8EE093E061
:103DD0000E94150E21E0019709F020E020930E01CA
:103DE00030E03E8B2D8BBE016B5E7F4F88E090E014
:103DF0000E94B71164EF71E080E090E00E94A001A2
:103E00008091BE019091BF01A091C001B091C1010C
:103E10008D8B9E8BAF8BB88F21E030E0809171014C
:103E200090917201029711F430E020E042E050E0FE
:103E3000BE016B5E7F4F8BE193E00E94150E892BD4
:103E400009F0A2C082E090E090937201809371012A
:103E500061E771E08AE090E00E94B71164EF71E0E1
:103E600080E090E00E94A00180E1E2ECF1E0DE0160
:103E7000559601900D928A95E1F780E1D1011D924E
:103E80008A95E9F7FE0175967F01510131014F01D5
:103E90000AE010E0BE01615D7F4FC8010E94DB11A6
:103EA000CFA4D8A8D401CD92DD924D01BE01655DAD
:103EB0007F4FC80144960E94DB11B1E0CB1AD108B4
:103EC0004BA55CA5E8E0CE16D10438F481E09A0158
:103ED000245C3F4F2937310508F080E0D3014D9332
:103EE0005D933D01811153C061E080E00E940C0AA6
:103EF00080915C05882309F46BC081E990E00E9401
:103F00003D0A68EE73E080E090E00E94A0010E940C
:103F1000D2016B017C01C0920706D0920806E092A4
:103F20000906F0920A068091850190918601892BFD
:103F3000B9F0809184058823A1F0409180055091CB
:103F400081056091820570918305411551056105D8
:103F5000710531F081E04C155D056E057F0508F0B7
:103F600080E080937F0580917E058823A1F10E94E7
:103F7000481180E090E0892B51F20E944B02882387
:103F800031F20E940000C3CF84E090E05DCF0E5F6D
:103F90001F4F0A31110509F07DCFA6E0B1E047E9D6
:103FA00054E085E190E08C0F9D1F4096F701208141
:103FB000F2E0EF0EF11C2D93F5012081F2E0AF0E3F
:103FC000B11CFA012193AF018E159F0579F78CCFB3
:103FD00084E890E094CF80917D05882339F080912A
:103FE00084058111C6CF0E94A310C3CF00917C0528
:103FF0000DAF002309F454C080918405811102C0E3
:104000000E94A310C0907901D0907A01E0907B01CA
:10401000F0907C0120E030E0A901C701B6010E94C8
:10402000B63220E030E040E05FE387FD34C0C701F6
:10403000B6010E9493300E9476316B017C011C1402
:104040001D041E041F040CF094CF80917A059091FA
:104050007B058C339105B4F0092E000CAA0BBB0B29
:104060008C199D09AE09BF09B7FF07C0B095A0958F
:10407000909581959F4FAF4FBF4F0397A105B10515
:104080000CF477CFC701B6010E94530BD0927B0589
:10409000C0927A056ECFC701B6010E949230CBCF95
:1040A0008091720581110DC00E94D20160936E054E
:1040B00070936F05809370059093710581E08093F4
:1040C000720580916E0590916F05A0917005B09179
:1040D00071050097A105B105A9F0C81AD90AEA0A25
:1040E000FB0A11EDC11617E0D106E104F10450F00E
:1040F0000E94BE0E10926E0510926F051092700510
:104100001092710502E010E0809123069091240640
:10411000DC01ED91FC910084F185E02D09951816E4
:1041200019060CF01EC18091230690912406DC0133
:10413000ED91FC910284F385E02D0995F82E87FD21
:1041400031C08091250690912606892B59F58091E2
:10415000340690913506892B29F520912C0680E8AC
:10416000820F8037F8F4822F8F7090E00196909341
:1041700032068093310640912F065091300631E08F
:104180004115510521F08417950709F030E030936F
:104190003306207F20932B06E1E0F0E0F093260623
:1041A000E0932506809125069091260681309105A1
:1041B00009F476C08230910509F494C0892B89F501
:1041C000FFEE9F2DFF1508F0907F90932B0680E85F
:1041D000890F803750F4F0922C062F2D2F702F5F0F
:1041E00030E0309332062093310620912F06309133
:1041F000300681E02115310541F0409131065091A2
:1042000032064217530709F080E080933306903E50
:1042100009F43FC048F4903931F1903BD1F1903826
:1042200069F1F0922A0670CF983F29F0D0F386E02A
:10423000890F8330B0F7E0914006F0914106309746
:1042400081F321E09B3F09F020E041E09C3F09F031
:1042500040E061E09A3F09F060E081E0983F09F0BA
:1042600080E00995DECF21E030E0309328062093EE
:1042700027063093260620932506D3CF10922806D2
:104280001092270681E090E0909326068093250601
:10429000C8CFA1E0B0E0B0932606A0932506C1CF19
:1042A00080912B06803919F058F4803869F4F7FCB6
:1042B0000BC01093260600932506F0922906B1CF75
:1042C000803B39F0803E99F3109226061092250625
:1042D000A8CFF7FCF9CFF092290610932606009399
:1042E00025069FCF80912B06803919F0E8F480389D
:1042F00059F7F7FCE9CF80913306209127063091DA
:104300002806232B11F0F1101CC0E0913806F09123
:1043100039068823C9F23097B9F24F2D60912906EA
:10432000809131060995D0CF803B91F0803E61F6B7
:1043300080913306882341F2E0913C06F0913D06DE
:10434000EACFE0913606F09137068111E4CFBCCF79
:1043500080913306E0913A06F0913B068111DBCF64
:10436000B3CF0091550510915605F801808580FD69
:1043700015C00E94D201D8011996CD90DD90ED9024
:10438000FC901C976C197D098E099F09609351055B
:10439000709352058093530590935405C090510536
:1043A000D0905205E0905305F0905405C8010E944A
:1043B0000405809150058111EFC0E0915505F09101
:1043C000560580858570853039F0B8ECCB16D10460
:1043D000E104F1040CF4E0C00E94D2016093660590
:1043E00070936705809368059093690580916505D2
:1043F000882309F4C2C00E94460F80916C059091F9
:104400006D056BE070E00E944433892BA1F484E1D8
:104410000E9469019C0191E02A3031050CF090E086
:1044200080917301981739F0909373012A30310508
:1044300014F40E94D41080916C0590916D0567E092
:1044400070E00E944433892BB9F5F090630100912C
:104450004C0510914D05D8011B968C91823008F0C7
:10446000E0C0F894C8010E947508F801E7807894CC
:10447000D0904B05ED1409F433C10E2D0E2C000C19
:10448000110B6091710170917201C8010E94443357
:10449000892B09F025C10E94D201609366057093B3
:1044A0006705809368059093690580916505882369
:1044B00009F4B9C00E94460F809185019091860150
:1044C000892B11F00C949B2C80916C0590916D05BB
:1044D00063E070E00E944433892B11F00C949B2C14
:1044E00085E10E94690120E034E0281B390B8091AE
:1044F000FE04082E000C990BFC01EE0FFF1FEC527E
:10450000FB4F31832083019665E170E00E944433C4
:104510008093FE0489010650110928961FAF0EAF43
:10452000289784ED94E00E94EF112A969FAF8EAFFA
:104530002A976C01F12CE12CC701B6010E94AC3125
:104540004B015C011091D30423961FAF23971111E7
:104550000C94EE2A8091FA0502E010E0882311F015
:1045600005E010E028968EAD9FAD2897863F9340DA
:1045700010F00C942D2B0C94F72A81E080935005B9
:1045800080918B018823F9F0E8ECCE16D104E10488
:10459000F104CCF40E94D41080915005882309F4D2
:1045A0002CCFE0915505F0915605808580FF25CFF1
:1045B0001092500510925105109252051092530519
:1045C000109254051ACF60E091E089270E941A11D9
:1045D00080918B018823D9F010924F0560E081E033
:1045E0000E94FF008091850190918601892B59F4EA
:1045F00010928100109285001092840080914E05E7
:1046000080618093810081E080935E05C5CF209119
:1046100085013091860181E021303105A9F380E0E8
:10462000F3CFF89422CF0D191109D7FC1395DD248F
:10463000D3941016110614F0DD24DA9480916301EE
:104640009091640100916F011091700197FD0CC071
:1046500027E0289FF001299FF00D1124E95FFA4F10
:1046600084819581892B91F40F3F100709F0A5C033
:1046700080916D0190916E01019609F09EC080912C
:1046800042058D0D87FF90C0825FFCCF0130110580
:1046900009F070C0EF2D0F2C000CFF0BED5BFA4FF3
:1046A0009081892F97FF02C08195D19401E0D012AB
:1046B00006C08A323CF4803144F0DD0C06C08B32F7
:1046C0000CF454C02D2D220FD20E8D0D8D330CF015
:1046D0008CE397FD819580830E947A0DE0924B05D3
:1046E00080914005909141050E940405E0914005AC
:1046F000F091410580858570853009F0DDCE0E94FE
:10470000D201609366057093670580936805909366
:104710006905809165058111CDCE809163019091ED
:10472000640197FD1BC027E0289FF001299FF00D31
:104730001124E95FFA4F84819581892B79F080916A
:104740006F0190917001019709F0D6C0EF2DFF0C19
:10475000FF0BED5BFA4F10820E947A0D80913F05AE
:10476000882309F4DAC010923F05A6CE81310CF4FB
:10477000ACCFA3CF80916D0190916E01019709F0AC
:10478000ADCFEF2D0F2C000CFF0BEB59FE4F8081AE
:104790008D0D89302CF088E080830E94560D9ECFCD
:1047A0001816D4F381E0F8CF082E000C990B6EE0B8
:1047B00070E00E944433809342051092060561E048
:1047C00080E00E940C0A0E94D2016093020570935F
:1047D0000305809304059093050520914205822FDF
:1047E000022E000C990B90930105809300050F3F5A
:1047F0001007E1F0B8016D0D711DD7FC7A95653099
:1048000071052CF477FF05C064E070E002C070E031
:1048100060E07093700160936F018DE992E00E94F7
:104820009B0E9093700180936F0158CF60916D0142
:1048300070916E016F3F7607D9F06D0D711DD7FC39
:104840007A95653071052CF477FF05C064E070E05F
:1048500002C070E060E070936E0160936D018FEABA
:1048600092E00E949B0E90936E0180936D0136CF73
:104870002730CCF483E293E00E94E80A809100059F
:10488000909101058730910508F028CF880F991F76
:10489000FC01E25FFD4F2DE044E061E08081918109
:1048A0000E94EB0D1BCF8C309105D9F461E080E0C4
:1048B0000E940C0A87E892E00E94E80A8091FF04B7
:1048C000882361F080E892E02DE04AE061E00E94F8
:1048D000EB0D61E080E00E940C0A00CF84E892E0DA
:1048E000F3CF880F991FFC01E25FFD4F2DE040E000
:1048F00061E080819181EBCF80916D0190916E019B
:10490000019709F02BCFEF2DFF0CFF0BEB59FE4F5A
:1049100081E080830E94560D21CF0E942812CCCDC9
:1049200094E0E916F10409F0D2C652C788E893E191
:10493000A0E0B0E022968CAF9DAFAEAFBFAF2297A4
:1049400047C7A70196012550310941095109A4E53E
:10495000B1E00E94173027EF33E040E050E00E94C2
:10496000F82FCA01B901675E7F4F8F4F9F4F0E949A
:10497000AE3120E030E040E05FE30E9493300E94DF
:10498000763122966CAF7DAF8EAF9FAF229769369E
:1049900071408105910554F008E611E020E030E017
:1049A00022960CAF1DAF2EAF3FAF229722968CAD53
:1049B0009DADAEADBFAD22974E97A105B1050CF0F0
:1049C00007C70EE110E020E030E022960CAF1DAFEB
:1049D0002EAF3FAF2297FCC6AB01BC018EEE95E037
:1049E0000E9487070E94E9310BC7C701B6010E94E8
:1049F000923049C72115310598E04907510560F407
:104A000082E080934E05C701B60120EA30E040E025
:104A100050E00E94613051C721153105A0E44A07DA
:104A2000510550F483E080934E05C701B60120E0A4
:104A300035E040E050E0EDCF211531054105B1E012
:104A40005B0750F484E080934E05C701B60120E077
:104A500034E140E050E0DDCF85E080934E05211544
:104A600031054105544038F4C701B60120E030E576
:104A700040E050E0CECF8FEF9FEF9093CE04809335
:104A8000CD041FC782E090E072C70E94BE0E20E1F5
:104A900040E061E080E393E00E94EB0D60918701CC
:104AA000709188018091890190918A010E94AE31B4
:104AB00020917401309175014091760150917701F8
:104AC0000E9404310E9476310E94530B77C70E94E6
:104AD000BE0E20E140E061E08BE393E00E94EB0D2D
:104AE0006DC720E140E061E086E493E0F7CF80917C
:104AF000B6059091B705A091B805B091B905892B7D
:104B00008A2B8B2B09F4C2C70E947B012091B6052A
:104B10003091B7054091B8055091B90564197509F0
:104B200086099709261737074807590708F0AEC7BF
:104B30008091B5050E943303F12C1092AB04F092E2
:104B4000AA0424968EAD9FAD2497F816190609F095
:104B500048C090E080E02496AEADBFAD24978A17A0
:104B60009B07C0F52896EEADFFAD28978181928115
:104B7000DC01ED91FC910284F385E02D0995809391
:104B8000EA0581E090E0E7CF35EE3093BC00D3C773
:104B90008091B6059091B705A091B805B091B9057F
:104BA000892B8A2B8B2B09F4CAC70E947B01209189
:104BB000B6053091B7054091B8055091B905641913
:104BC000750986099709261737074807590708F016
:104BD000B6C7AECF2A96EEADFFAD2A97EF2B09F4FC
:104BE00032C7D8014D915D916D917C914115510570
:104BF0006105710541F0D501C401841B950BA60B1D
:104C0000B70BAC01BD01D80114968D919C911597FD
:104C10002091EA0530E00C2C02C0359527950A94C6
:104C2000E2F720FD1BC1009709F0F2C0F801808275
:104C30009182A282B38221E030E0358324832FEF7A
:104C4000C21AD20A095F1F4F38E0C316D10409F017
:104C5000F2C60DAD002309F44DC0F0906301F7FCDE
:104C600040C00F2D0F2C000C110B27E0F0E0E0E00E
:104C70002F153CF03F2D47E03402F0011124E55F91
:104C8000FA4F808191818330910509F40FC1049717
:104C900041F580918B01811124C08091060581111D
:104CA00020C080916F019091700197FF1AC0809190
:104CB0006D0190916E0197FF14C060E080E00E944A
:104CC0000C0A84EA90E00E943D0AC80101960E9405
:104CD000C10A8FE990E00E943D0AF09280010E9493
:104CE000930580916B05811105C080916A05811142
:104CF00010926A0580916C0590916D0501969093D4
:104D00006D0580936C0560E177E20E944433892B46
:104D1000A9F480918B01882309F44AC28091070687
:104D200090910806A0910906B0910A068093660545
:104D300090936705A0936805B09369058091650518
:104D4000882309F45DC0C0905F05D0906005E090B5
:104D50006105F09062058091070690910806A09188
:104D60000906B0910A068C199D09AE09BF0985365E
:104D70009105A105B10508F443C0009163051091A8
:104D8000640560E0802F0E940C0A60E28BE096E0F0
:104D90000E941B0A8FE0B82E61E08B2D801B0E94C1
:104DA0000C0A60E28BE096E00E941B0AC8010196A3
:104DB00060E170E00E944433182F80936305909364
:104DC000640560E00E940C0A6FEF8BE096E00E94A1
:104DD0001B0A61E08B2D811B0E940C0A6FEF8BE098
:104DE00096E00E941B0A14E6C10ED11CE11CF11CC6
:104DF000C0925F05D0926005E0926105F092620575
:104E000080915E05882309F405C210925D05B1C842
:104E10008130910599F4453151056105710508F41A
:104E20000ECF82E090E015969C938E931497D092CB
:104E30006401C0926301B1E0BDAF01CF029709F0F8
:104E4000FECE493E53406105710508F4F8CE84E07A
:104E500090E015969C938E931497EDCF8230910538
:104E6000E9F08430910569F0019709F0E8CE453109
:104E700051056105710508F4E2CEF801158214822E
:104E8000DECE15961C921E92149716961C928FEFEA
:104E90009FEF9093640180936301CDCF83E090E016
:104EA000F80195838483F1E0FDAFC9CE80916F0155
:104EB00090917001019709F412CF80916D0190914A
:104EC0006E01019709F40BCF80910605882309F440
:104ED00011C10E947B012B013C018091A2049091A1
:104EE000A304A091A404B091A5040097A105B10565
:104EF00009F491C04091A6045091A7046091A804C0
:104F00007091A904411551056105710509F483C02B
:104F10008C019D01041B150B260B370BB901A80151
:104F200073016201C81AD90AEA0AFB0AC416D50637
:104F3000E606F70610F468017901C701B6010E9480
:104F4000AC319B01AC0160E070E68AE697E40E9418
:104F5000043120E030E04AE754E40E94BB320E9472
:104F600076319B012E5131092B33324008F0B9C004
:104F7000072E000C880B990B0E94AE314B015C018F
:104F80008092790190927A01A0927B01B0927C018B
:104F900020E030E0A9010E94B63220E030E040E09D
:104FA0005FE387FD51C0C501B4010E9493300E94A8
:104FB00076310E94530BC701B60124EB30E040E08C
:104FC00050E00E946130A0EAB0E00E9417306B010F
:104FD0007C0124E130E040E050E00E946130211586
:104FE000310581E048075105A0F581E080934E0529
:104FF0003093CE042093CD048091CD049091CE04C3
:10500000909387008093860080914E058061809305
:1050100081000E9448118091A2049091A304A09164
:10502000A404B091A5048093A6049093A704A09330
:10503000A804B093A9044092A2045092A3046092E1
:10504000A4047092A5044BCEC501B4010E94923015
:10505000AECF2115310598E04907510560F482E093
:1050600080934E05C701B60120EA30E040E050E0F1
:105070000E946130BDCF21153105A0E44A075105DA
:1050800050F483E080934E05C701B60120E035E07F
:1050900040E050E0EDCF211531054105B1E05B075F
:1050A00050F484E080934E05C701B60120E034E15E
:1050B00040E050E0DDCF85E080934E0521153105BD
:1050C0004105544038F4C701B60120E030E540E026
:1050D00050E0CECF8FEF9FEF9093CE048093CD041E
:1050E0008BCF1092A2041092A3041092A4041092E9
:1050F000A50491CFE0914005F0914105808580FDA8
:1051000004C08F2D0E94E30BEACD80916B058823AC
:10511000F9F0F6E0FF15D4F0F3948091A1048F1517
:1051200091F0F092A1048F2DFF0C990B9093300613
:1051300080932F069A838983BE016F5F7F4F82E041
:1051400090E00E94B7110E94BE0EC9CDF12CE5CFB0
:105150008091A004882301F180916A058111BFCD5F
:105160008091840180310CF0BACD91E090936A0572
:1051700061E00E940C0AC80101960E94C10AE091F8
:10518000840181E08E0F809384010E2E000CFF0BB2
:10519000E358FE4FF78AA3CD80917D0190917E0167
:1051A000069709F49CCD81E08F0D0E94CC0D97CD20
:1051B000809165058111C7CD0E94D20100916605DD
:1051C000109167052091680530916905601B710B8E
:1051D000820B930B613E73498440910508F410CE15
:1051E00081E08093650510926405109263058091BB
:1051F000070690910806A0910906B0910A068093CF
:105200005F0590936005A0936105B09362050E94CD
:10521000630994CD80917C0581110C94B91F809114
:105220008B01811106C080916B05882311F40C94C9
:10523000B91F80915D05882309F45EC000915C056B
:10524000002349F080E10E94D600892B21F461E01F
:1052500080E10E94FF0010925D0581E080935B0574
:1052600080916B05882309F4A6C01091780160E055
:10527000812F0E94FA0A809162018F3009F08BC061
:10528000E2E5F1E081E691E0218121938E179F070D
:10529000D9F7E09162010E2E000CFF0BEE5AFE4F83
:1052A00010830E94D2010091020510910305209104
:1052B000040530910505601B710B820B930B693B54
:1052C0007B4081059105C0F061E080E00E940C0AFE
:1052D00002E511E0F12CD8016D918D0167FD66C0EA
:1052E000809162018F115BC08BE096E00E941B0AE7
:1052F000F394B0E1FB12EFCF6091870170918801C8
:105300008091890190918A0122E030E040E050E0F4
:105310000E94F82FCA01B9010E94AE312091740198
:105320003091750140917601509177010E940431CE
:1053300020E030E44CE955E40E94B63208EC10E07D
:10534000181614F008EE13E080915B05882311F421
:105350000C94B91F0E947B01012E000C220B330B11
:10536000C0905705D0905805E0905905F0905A0527
:105370000C0D1D1D2E1D3F1D601771078207930721
:1053800010F40C94B91F10925B0560E083E00E945A
:10539000FF000C94B91F8F5F809362017ACF862F34
:1053A000660F990B01960E94C10AA2CF82E792E094
:1053B0000E94E80A9DCFF0907F0180919F04815068
:1053C00080939F041091800118160CF494C02091D2
:1053D0007D0130917E012330310509F4BEC0C0F457
:1053E000109180012130310509F46FC02230310560
:1053F00009F494C0109180011F5F1F150CF0B9C013
:10540000002309F479C001E0112309F475C073C0C9
:105410002530310509F4D3C008F4B6C02630310573
:1054200049F70E94D20100910205109103052091D5
:105430000405309105056B017C01C01AD10AE20A0E
:10544000F30A80918301082F082E000C110BB9EB91
:10545000CB16BBE0DB06E104F10468F061E00E94DA
:105460000C0AF801E358FE4F8789082E000C990BAF
:1054700001960E94C10A80918301082E000C990BAD
:10548000019660918401062E000C770B0E94443334
:1054900080938301FC01E358FE4F178900915C055E
:1054A000002319F001E0811100E0E9EBCE16EBE0FA
:1054B000DE06E104F10400F161E00E940C0A612FB4
:1054C0008BE096E00E941B0A17C0115017FD02C026
:1054D0001F1514F01FEF1F0D002371F06F2DFF0C2F
:1054E000770B6150710901E0812F012E000C990B9F
:1054F0006817790709F000E0602F812F0E94FA0AEF
:1055000080919F0418160CF4F7CEE12F110FFF0BBA
:10551000EB59FE4F808180939F04EECE80918101F4
:10552000882359F01F5F17FF0AC081E08093810133
:10553000011111C000E010E0DFCF1150F4CF1F15B2
:105540002CF01FEF1F0D10928101D5CF0023A1F287
:10555000882389F258CF10E056CFE1E0FE1609F417
:1055600006C38091800112E0180F1F152CF080FFF8
:1055700032C00111E0CFDECF002309F4BDCF01E03E
:10558000112309F4B9CFB7CF80918201082E000C06
:10559000990B01966F2DFF0C770B0E944433282F37
:1055A0008093820183589E4FDC011F961C9100233B
:1055B00009F4A2CF01E0222309F49ECF9CCF0E94E0
:1055C000BE2F892F990F990B6F2DFF0C770B0E941F
:1055D0004433182F90CF00E011E08ECF28960EAD07
:1055E0001FAD2897063F134068F502E310E02091B5
:1055F000CF043091D0044091D1045091D204C50120
:10560000B4010E9492302B013C0120E030E0A9015E
:105610000E94B632181624F077FA709477F87094D6
:10562000B801110F880B990B0E94AE31A3019201B2
:105630000E94B63218160CF47EC123960FAD239744
:10564000002359F020E140E061E088E293E00E940D
:10565000EB0D1092D304109206058092CF04909225
:10566000D004A092D104B092D2048091FA0588238C
:1056700009F467C98AE0E2EDF1E0DE015596019098
:105680000D928A95E1F784E1ECEDF1E0DE011196EF
:1056900001900D928A95E1F720E030E040EA50E475
:1056A000C501B4010E94FF3087FD8BC920E030E4C2
:1056B0004EE754E4C501B4010E94B63218160CF44A
:1056C00035C96E0117E1C10ED11CF12CE12C870107
:1056D0002FEFE21AF20AD6012D913D916D01C90119
:1056E000330FAA0BBB0B26968CAF9DAFAEAFBFAFEF
:1056F0002697BC01CD010E94AE319B01AC01C501D2
:10570000B4010E94FF3087FF0BC9EE0CFF1CEE0CAA
:10571000FF1CF101EE0DFF1D80809180A280B380FF
:10572000F801EE0FFF1FEE0FFF1FE20DF31D60816A
:105730007181828193810E94AE310E9476312B016A
:105740003C01000F111FF101E00FF11FC488D58843
:105750000D2C000CEE08FF08C501B4010E94AE310B
:105760000E9476319B01AC0124193509460957097D
:105770002A960EAD1FAD2A97B80190E080E06C1913
:105780007D098E099F090E94283326962CAD3DADD8
:105790004EAD5FAD26972C193D094E095F090E9459
:1057A000F82FDA01C901840D951DA61DB71D22969B
:1057B0008CAF9DAFAEAFBFAF229788169906AA06F1
:1057C000BB0634F422968CAE9DAEAEAEBFAE229731
:1057D00022966CAD7DAD8EAD9FAD22970E94AE310D
:1057E00028960EAD1FAD2897063F134008F4F4C865
:1057F0006093F2057093F3058093F4059093F5059B
:105800000E947631009187011091880120918901D1
:1058100030918A01061717072807390709F47CC059
:1058200060938701709388018093890190938A0126
:105830000E94AE319B01AC0160EC71EE84E69CE409
:105840000E940431209174013091750140917601DC
:10585000509177010E94BB3220E030E044E353E4F2
:105860000E9404316B017C0120E030E0A9010E941C
:10587000B63220E030E040E05FE387FDB6C8C70104
:10588000B6010E9493300E947631A0EAB0E09B01FD
:10589000AC010E9417306B017C0124E130E040E054
:1058A00050E00E9461302115310581E04807510523
:1058B00008F0A0C881E080934E053093CE04209379
:1058C000CD048091CD049091CE0490938700809375
:1058D000860080914E0580618093810080918501D2
:1058E00090918601892BC1F46091870170918801A4
:1058F0008091890190918A010E94AE3120917401BA
:105900003091750140917601509177010E940431E8
:105910000E9476310E94530B0E94D201609366056B
:10592000709367058093680590936905809165057C
:1059300081110E94460F80916C0590916D056FED6D
:1059400073E00E944433892B09F063C08EE00E940B
:10595000D600182F81E10E94D600112309F492C8C5
:1059600031E020E0811101C030E0832F922F20919F
:105970008501309186012817390709F44AC0109231
:10598000D3041092060590938601809385011092AE
:105990004F0560E081E00E94FF0060E083E00E942C
:1059A000FF0080918501909186018130910509F475
:1059B0008EC808F46AC8029709F493C880E00E9470
:1059C00006128091850190918601892B81F080914A
:1059D000CC0481110DC08091FF04882349F02091EF
:1059E00085013091860181E02130310509F080E0A8
:1059F000809384050E94D2016093660570936705C9
:105A000080936805909369058091650581110E94D6
:105A1000460F80916C0590916D056FE170E00E94DA
:105A200044336C01892B09F065C90E94D2014B01F6
:105A30005C0107E015E02091EC053091ED0528961A
:105A40003FAF2EAF28972896AEADBFAD28971496DE
:105A50000D90BC91A02D2A96BFAFAEAF2A97EE2431
:105A6000E394AB2B09F4E12CEE2DF0E02496FFAF8C
:105A7000EEAF24972896AEADBFAD2897BC912B967C
:105A8000BFAF2B970E947B012B013C018091B40595
:105A900081112DC8FE2CE1E0E093B405E092B3053E
:105AA000FFEFF093B2051092B1058FEF8E0D80934A
:105AB000B005E0938F0580918F052B969FAD2B97B6
:105AC000990F892B80938F0580918E05813009F085
:105AD0005BC810928E050E947B012B013C018091D6
:105AE0008F058093BB008091B6059091B705A0917A
:105AF000B805B091B905892B8A2B8B2BA9F00E9490
:105B00007B012091B6053091B7054091B8055091C1
:105B1000B9056419750986099709261737074807D3
:105B2000590710F40C9498258091BC0083FDD7CFC1
:105B300025EC2093BC000E947B012B013C0180914D
:105B4000B405813009F424C88091B1058E1510F494
:105B5000F090B105A0E9B5E0ECEAF4E080E08F1543
:105B600011F40C949D259D9191938F5FF8CF0023A4
:105B700009F4E1CC01E0DFCCCF93DF93DC012D9180
:105B8000FB013191EC013883EB012883415051092D
:105B9000CD01BF01141615068CF3DF91CF91089546
:105BA000B0E0A0E0E6EDFDE20C9434306C01D62FBD
:105BB000C72F8A017901F9010995B80197FF15C02E
:105BC0008D2F9C2FF701099597FD08C0B801C601DC
:105BD000F701099597FD16C0DC2DCD2D8D2F9C2F3B
:105BE000CDB7DEB7E8E00C9450308D2F9C2FF70135
:105BF00009951816190694F3B801C601F70109951D
:105C000097FDEACFD02FC12FE9CFA8E0B0E0EBE0BD
:105C1000FEE20C942A308C0158874F8359019A0177
:105C20003195219531093E832D836F807884600EF4
:105C3000711E6730710578F58F819885689F6001C6
:105C4000699FD00C789FD00C1124C00ED11E6C140B
:105C50007D0420F02896E2E10C944630730113C0D5
:105C600047012F813885821A930AB701C401F501D3
:105C700009951816190654F44F815885B401C701C7
:105C80000E94BC2D74010E151F0550F3EF81F8859D
:105C90006E0E7F1EDCCFCB01969587952F813885C0
:105CA000829F6001839FD00C929FD00C1124C00E64
:105CB000D11ECB010197829F1001839F300C929FD0
:105CC000300C11247801E20CF31C6730710509F4E3
:105CD00042C0C701280169327105B0F183E07695B1
:105CE00067958A95E1F7629F4001639F900C729FD0
:105CF000900C1124C401880F991F9A838983AC01E9
:105D0000400F511FB801680D791D9501C8010E940F
:105D1000D02D2C01A601480D591D91948194910814
:105D20009501B601C601880D991D0E94D02D6C0108
:105D3000B701680D791D9501A701C701E981FA81B5
:105D40008E1B9F0B0E94D02D9501AC01B601C201A4
:105D50000E94D02D6C014F815885B601C8010E9468
:105D6000BC2D4301630127011A821982EC14FD0442
:105D700008F446C0B801C601F501099518161906C0
:105D800054F1892B71F44F815885B601C3010E94EB
:105D9000BC2D2F813885620E731E81E090E09A83BE
:105DA0008983EF81F885CE0EDF1EE0CF892B71F459
:105DB0004F815885B201C7010E94BC2D2D813E81C3
:105DC000420E531E81E090E09A838983EB80FC8031
:105DD000EC14FD04A8F0B801C701F50109952D8167
:105DE0003E812E0D3F1D3C832B8397FFDFCF4F81DC
:105DF0005885B701C6010E94BC2DEB80FC80CDCF39
:105E0000EF81F8852E0E3F1E200E311E29813A812A
:105E1000232B09F58214930408F01CCF740113C0DE
:105E20006701EF81F885CE1ADF0AB701C601F501D7
:105E300009951816190654F44F815885B601C70103
:105E40000E94BC2D76010E151F0550F38F81988599
:105E5000880E991EDFCF460186189708A301401BC4
:105E6000510B841695060CF4A4011416150634F48F
:105E7000B601641B750BC8010E94BC2D92012E193E
:105E80003F097901A101441955098F819885481B63
:105E9000590B2417350708F4A9011416150634F414
:105EA000B101641B750BC6010E94BC2DEF81F88502
:105EB000E815F90548F4C401BF010E94E42F9501DB
:105EC000AF01C8010E94052E2F8138852E153F0590
:105ED00008F0C0CE81010E191F09C701B9010E9447
:105EE000E42FA3CE8F929F92AF92BF92CF92DF9278
:105EF000EF92FF92CF93DF93EC01688179818A81E1
:105F00009B81611571058105910521F464E279EDAC
:105F10008BE597E02DE133EF41E050E00E94F82F50
:105F200049015A019B01AC01A7EAB1E40E94173074
:105F30006B017C01ACEEB4EFA50194010E94253009
:105F4000DC01CB018C0D9D1DAE1DBF1DB7FF03C035
:105F50000197A109B04888839983AA83BB839F775F
:105F6000DF91CF91FF90EF90DF90CF90BF90AF90F7
:105F70009F908F9008950E94722F089584EA91E077
:105F80000E94722F0895B0E0A0E08093A401909346
:105F9000A501A093A601B093A7010895F999FECF9A
:105FA00092BD81BDF89A992780B50895262FF99959
:105FB000FECF1FBA92BD81BD20BD0FB6F894FA9AEC
:105FC000F99A0FBE01960895AA1BBB1B51E107C0A9
:105FD000AA1FBB1FA617B70710F0A61BB70B881F79
:105FE000991F5A95A9F780959095BC01CD01089508
:105FF000052E97FB1EF400940E940F3057FD07D02A
:106000000E94613007FC03D04EF40C940F30509581
:106010004095309521953F4F4F4F5F4F0895909594
:106020008095709561957F4F8F4F9F4F08950E9487
:106030008330A59F900DB49F900DA49F800D911D5E
:1060400011240895B7FF0C9417300E941730821B5B
:10605000930B08952F923F924F925F926F927F928F
:106060008F929F92AF92BF92CF92DF92EF92FF9268
:106070000F931F93CF93DF93CDB7DEB7CA1BDB0B14
:106080000FB6F894DEBF0FBECDBF09942A883988B9
:1060900048885F846E847D848C849B84AA84B984C0
:1060A000C884DF80EE80FD800C811B81AA81B981CC
:1060B000CE0FD11D0FB6F894DEBF0FBECDBFED01E0
:1060C0000895A1E21A2EAA1BBB1BFD010DC0AA1F39
:1060D000BB1FEE1FFF1FA217B307E407F50720F051
:1060E000A21BB30BE40BF50B661F771F881F991FCC
:1060F0001A9469F760957095809590959B01AC0115
:10610000BD01CF010895A29FB001B39FC001A39F1D
:10611000700D811D1124911DB29F700D811D1124E0
:10612000911D08955058BB27AA270E94AA300C94AD
:1061300064320E94563238F00E945D3220F039F409
:106140009F3F19F426F40C9453320EF4E095E7FBCC
:106150000C942432E92F0E94753258F3BA17620763
:1061600073078407950720F079F4A6F50C94AF32F5
:106170000EF4E0950B2EBA2FA02D0B01B901900162
:106180000C01CA01A0011124FF27591B99F0593FA6
:1061900050F4503E68F11A16F040A22F232F342FEE
:1061A0004427585FF3CF469537952795A795F0403C
:1061B0005395C9F77EF41F16BA0B620B730B840B51
:1061C000BAF09150A1F0FF0FBB1F661F771F881F09
:1061D000C2F70EC0BA0F621F731F841F48F4879561
:1061E00077956795B795F7959E3F08F0B0CF939553
:1061F000880F08F09927EE0F9795879508950E94CC
:10620000003208F481E008950E9418310C94643241
:106210000E945D3258F00E94563240F029F45F3FF0
:1062200029F00C94243251110C94B0320C94533256
:106230000E94753268F39923B1F3552391F3951BAE
:10624000550BBB27AA2762177307840738F09F5F97
:106250005F4F220F331F441FAA1FA9F335D00E2E04
:106260003AF0E0E832D091505040E695001CCAF771
:106270002BD0FE2F29D0660F771F881FBB1F261734
:1062800037074807AB07B0E809F0BB0B802DBF010B
:10629000FF2793585F4F3AF09E3F510578F00C94DA
:1062A00024320C94B0325F3FE4F3983ED4F38695E9
:1062B00077956795B795F7959F5FC9F7880F911DFB
:1062C0009695879597F90895E1E0660F771F881FE7
:1062D000BB1F621773078407BA0720F0621B730B9A
:1062E000840BBA0BEE1F88F7E09508950E947D316C
:1062F0006894B1110C94B03208950E947D3288F0F8
:106300009F5798F0B92F9927B751B0F0E1F0660F79
:10631000771F881F991F1AF0BA95C9F714C0B130BA
:1063200091F00E94AF32B1E008950C94AF32672F24
:10633000782F8827B85F39F0B93FCCF386957795E9
:106340006795B395D9F73EF49095809570956195D2
:106350007F4F8F4F9F4F0895E89409C097FB3EF4FD
:1063600090958095709561957F4F8F4F9F4F9923A2
:10637000A9F0F92F96E9BB279395F6958795779520
:106380006795B795F111F8CFFAF4BB0F11F460FFE0
:106390001BC06F5F7F4F8F4F9F4F16C0882311F038
:1063A00096E911C0772321F09EE8872F762F05C04C
:1063B000662371F096E8862F70E060E02AF09A95E7
:1063C000660F771F881FDAF7880F9695879597F9DC
:1063D00008950E94973290F09F3748F4911116F07B
:1063E0000C94B03260E070E080E89FEB089526F4F2
:1063F0001B16611D711D811D0C942A320C944532AF
:10640000990F0008550FAA0BE0E8FEEF16161706C5
:10641000E807F907C0F012161306E407F50798F02D
:10642000621B730B840B950B39F40A2661F0232B46
:10643000242B252B21F408950A2609F4A140A695C2
:106440008FEF811D811D089597F99F6780E870E0A7
:1064500060E00895882371F4772321F09850872B0A
:10646000762F07C0662311F499270DC09051862B13
:1064700070E060E02AF09A95660F771F881FDAF7C0
:10648000880F9695879597F908959F3F31F0915021
:1064900020F4879577956795B795880F911D969508
:1064A000879597F908959FEF80EC089500240A944A
:1064B0001616170618060906089500240A941216DF
:1064C0001306140605060895092E0394000C11F412
:1064D000882352F0BB0F40F4BF2B11F460FF04C0BF
:1064E0006F5F7F4F8F4F9F4F089557FD9058440F18
:1064F000551F59F05F3F71F04795880F97FB991F23
:1065000061F09F3F79F087950895121613061406DF
:10651000551FF2CF4695F1DF08C01616170618066C
:10652000991FF1CF869571056105089408950E9421
:106530007D32A0F0BEE7B91788F4BB279F3860F41E
:106540001616B11D672F782F8827985FF7CF86958D
:1065500077956795B11D93959639C8F30895E8949A
:10656000BB2766277727CB0197F908950E94003251
:1065700008F48FEF08950E94CE320C9464320E948A
:10658000563238F00E945D3220F0952311F00C94C1
:1065900024320C94533211240C94B0320E94753280
:1065A00070F3959FC1F3950F50E0551F629FF00166
:1065B000729FBB27F00DB11D639FAA27F00DB11D7F
:1065C000AA1F649F6627B00DA11D661F829F222708
:1065D000B00DA11D621F739FB00DA11D621F839F8F
:1065E000A00D611D221F749F3327A00D611D231F65
:1065F000849F600D211D822F762F6A2F11249F57B3
:1066000050409AF0F1F088234AF0EE0FFF1FBB1FB5
:10661000661F771F881F91505040A9F79E3F510574
:1066200080F00C9424320C94B0325F3FE4F3983E37
:10663000D4F3869577956795B795F795E7959F5F1E
:10664000C1F7FE2B880F911D9695879597F90895B0
:10665000DB018F939F930E941730BF91AF91A29F50
:10666000800D911DA39F900DB29F900D1124089550
:10667000991B79E004C0991F961708F0961B881F94
:106680007A95C9F78095089597FB072E16F4009424
:1066900007D077FD09D00E94E42F07FC05D03EF417
:1066A000909581959F4F0895709561957F4F0895BE
:1066B0000E948330B7FF0895821B930B0895EE0F5D
:1066C000FF1F0590F491E02D09940F931F93CF9332
:1066D000DF938230910510F482E090E0E091F506BE
:1066E000F091F60630E020E0B0E0A0E0309799F4B9
:1066F0002115310509F44AC0281B390B2430310516
:10670000D8F58A819B816115710589F1FB0193831D
:106710008283FE0111C0408151810281138148179B
:106720005907E0F04817590799F4109761F012964D
:106730000C93129713961C933296CF01DF91CF9151
:106740001F910F9108950093F5061093F606F4CF6C
:106750002115310551F04217530738F0A901DB012B
:106760009A01BD01DF01F801C1CFEF01F9CF90938C
:10677000F6068093F506CDCFFE01E20FF31F81935D
:1067800091932250310939832883D7CF2091F30682
:106790003091F406232B41F42091AA013091AB01F2
:1067A0003093F4062093F3062091A8013091A901BB
:1067B0002115310541F42DB73EB74091AC01509100
:1067C000AD01241B350BE091F306F091F406E217BE
:1067D000F307A0F42E1B3F0B2817390778F0AC0104
:1067E0004E5F5F4F2417350748F04E0F5F1F5093E1
:1067F000F4064093F306819391939FCFF0E0E0E09D
:106800009CCFCF93DF930097E9F0FC01329713827E
:106810001282A091F506B091F606ED0130E020E07D
:106820001097A1F420813181820F931F2091F306EC
:106830003091F4062817390709F061C0F093F40687
:10684000E093F306DF91CF910895EA01CE17DF07B9
:10685000E8F54A815B819E0141155105B1F7E901D7
:10686000FB83EA8349915991C40FD51FEC17FD07AB
:1068700061F4808191810296840F951FE9019983CB
:106880008883828193819B838A83F0E0E0E0129683
:106890008D919C9113970097B9F52D913C9111978B
:1068A000CD010296820F931F2091F3063091F406DA
:1068B0002817390739F6309751F51092F6061092DD
:1068C000F506B093F406A093F306BCCFD383C2833E
:1068D00040815181840F951FC817D90761F44E5F1D
:1068E0005F4F88819981480F591F518340838A8166
:1068F0009B81938382832115310509F0B0CFF093FA
:10690000F606E093F5069ECFFD01DC01C0CF1382B1
:106910001282D7CF81E090E0F8940C948F34F894F1
:02692000FFCFA7
:10692200B400E001E00101010101010101010118CE
:106932000305110E0E110E0E111F001E1D1B17173F
:10694200171F19170F010E0E111F000F011E1E0E29
:10695200111F1D19150D001D1D1F001D1B1D1E0ED3
:10696200111F110E1E1D1B17001F1B131B1B1B1BB0
:10697200111FFFFFFFFFFFFFFFFFFFFFFFFFFFFFF3
:10698200FFFFFFFFFF0101010101010101FFFFFF05
:10699200FF0200010000803FFF00004843000008A2
:1069A2000001000010000078000000000001020356
:1069B200040506070001020300010203040506079D
:1069C20004030201010000000000F7068000180025
:1069D2000C0006008002840252035503580356033A
:1069E2005303010001000100010001000100010048
:1069F2000100000080010003800300041E0000006B
:106A02007A00000072010000E80300008813000011
:106A1200A9025A035E0363036B0300FF01FF020333
:106A2200FF04FF05060700000000890585057203C3
:106A320079038103880391039903A603A003AD039D
:106A4200B703C203CC03D203D803000000008102C3
:106A5200E1010E02CE023F021D02310200000000DF
:106A6200D404A704C4087D04A0048D047E0400009D
:106A720000001B0AE101C408C30800000000F3077C
:106A8200E101C408C3086A085F08F60701085B0051
:106A920020202020002D00202B00202030002A0062
:106AA2006F6666006F6E00536574207377696E6758
:106AB200200053746570203120736574004D696342
:106AC200726F74696D696E6700436C656172004D27
:106AD200756C74697374657000496E7420636C6FB1
:106AE200636B206F6E6C79005374617274207461F1
:106AF200707300456E642074617073004446414DAA
:106B0200205468696E672020205B385D00416C74F8
:106B12002052756E206F75747075740053757070A5
:106B22006F72742066617374005050514E004B6551
:106B32007953746570204D49444900456E636F6412
:106B42006572005365742000456E642074617000A4
:106B5200496E742E20436C6F636B004578742E204F
:106B6200436C6F636B004D4944492E20436C6F6345
:106B72006B003234003132003600536574005361C9
:106B8200766500526573746F726500526574757232
:106B92006E004E6F726D616C005265766572736540
:106BA20000426F756E6365004F64642F4576656EB3
:106BB2000053687566666C650052616E646F6D00A5
:106BC200456E74657220437573746F6D004D494450
:106BD20049204D6F6465005365742073746570209D
:106BE20031005461702074656D706F004D756C7466
:0E6BF20069005377696E67004D6963726F002A
:00000001FF
